:100000000C94CC030C94E9030C9494220C94E90313
:100010000C94E9030C94E9030C94E9030C94E903B0
:100020000C94E9030C941A380C94E9030C94E9033A
:100030000C94E9030C94E9030C94E9030C94E90390
:100040000C94E9030C94E9030C94E9030C94E90380
:100050000C94E9030C945F440C94E9030C94E903B9
:100060000C94E9030C94E9030C94E9030C94E90360
:100070000C94E9030C94E9030C94E9030C94E90350
:100080000C94E9030C94E9030C94E9030C94E90340
:100090000C94E9039F39EA39A53ACA3A3E3B5F3BE3
:1000A000833B863B953BC541C541C541C541C541E3
:1000B000C541C541C541C541C541C541C541C54110
:1000C000C541C541C541C541C541C541C541C54100
:1000D000C541223CA43BBF3B403C503CC541C541CF
:1000E000C43D063E423E813EC541C541C541C54174
:1000F000C541C541C541C541C541C541C541C541D0
:10010000C541C541C541C541C541C541C541C541BF
:10011000C5417F3CC43CBA3ED33E033F1A3FC54174
:10012000C541C541C541C541C541C541C541C5419F
:10013000C541F43C4C3D273FA73F2640684007415E
:100140001641DF40F340254137414A41C5415B41FB
:10015000313D593D813D8F41AA41A940C440CE0364
:10016000C103B303A30390037A0361034703290385
:100170000803E602C2029E0276024F022802030230
:100180006C01B80196017501560139011F01060184
:10019000EF00DA00B5008200A500960000004341A0
:1001A0004E20310000000000000000000043414EDE
:1001B00020320000000000000000000043414E20FB
:1001C000330000000000000000000043414E2034D6
:1001D0000000000000000000000043414E203500F8
:1001E00000000000000000000043414E20360000E7
:1001F000000000000000000043414E2037000000D6
:100200000000000000000043414E203800000000C4
:1002100000000000000043414E20390000000000B3
:10022000000000000043414E20313000000000007B
:100230000000000043414E2031310000000000006A
:1002400000000043414E2031320000000000000059
:10025000000043414E203133000000000000000048
:100260000043414E20313400000000000000000037
:1002700043414E20313500000000000000000043E3
:10028000414E2031360000000000000000004341D4
:100290004E20313700000000000000000043414EB6
:1002A00020313800000000000000000043414E20D3
:1002B000313900000000000000000043414E2032B0
:1002C0003000000000000000000043414E203231A9
:1002D00000000000000000000043414E20323200C8
:1002E000000000000000000043414E2032330000B7
:1002F0000000000000000043414E203234000000A6
:1003000000000000000043414E2032350000000094
:10031000000000000043414E203236000000000083
:100320000000000043414E20323700000000000072
:1003300000000043414E2032380000000000000061
:10034000000043414E203239000000000000000050
:100350000043414E20333000000000000000000048
:1003600043414E20333100000000000000000043F4
:10037000414E203332000000000000000000466CB7
:1003800061736820310000000000000000466C61CD
:10039000736820320000000000000000466C6173AA
:1003A0006820330000000000000000466C617368A4
:1003B00020340000000000000000466C61736820DB
:1003C0003500000000000000005357495443482006
:1003D00031000000000000005357495443482032C8
:1003E00000000000000000535749544348203300E8
:1003F00000000000000053574954434820340000D7
:1004000000000000005357495443482035000000C5
:1004100000000000535749544348203600000000B4
:1004200000000053574954434820370000000000A3
:100430000000535749544348203800000000000092
:100440000053574954434820390000000000000081
:1004500053574954434820313000000000000053F6
:100460005749544348203131000000000000434800
:10047000414E4E454C2031000000000000434841F1
:100480004E4E454C20320000000000004348414ED3
:100490004E454C20330000000000004348414E4EC2
:1004A000454C20340000000000004348414E4E45BA
:1004B0004C20350000000000004348414E4E454CA2
:1004C00020360000000000004348414E4E454C20BD
:1004D000370000000000004348414E4E454C203894
:1004E0000000000000004348414E4E454C203900BA
:1004F00000000000004348414E4E454C2031300082
:10050000000000004348414E4E454C203131000070
:100510000000004348414E4E454C2031320000005F
:1005200000004348414E4E454C203133000000004E
:10053000004348414E4E454C20313400000000003D
:100540004348414E4E454C203135000000000043E9
:1005500048414E4E454C20313600000000004348D3
:10056000414E4E454C2031370000000000434841C9
:100570004E4E454C20313800000000004348414EAB
:100580004E454C20313900000000004348414E4E9A
:10059000454C20323000000000004348414E4E459B
:1005A0004C20323100000000004348414E4E454C83
:1005B00020323200000000004348414E4E454C209E
:1005C000323300000000004348414E4E454C20327B
:1005D0003400000000004348414E4E454C20323567
:1005E00000000000004348414E4E454C203236008A
:1005F000000000004348414E4E454C203237000079
:100600000000004348414E4E454C20323800000067
:1006100000004348414E4E454C2032390000000056
:10062000004348414E4E454C20333000000000004E
:100630004348414E4E454C203331000000000043FA
:1006400048414E4E454C20333200000000004348E4
:10065000414E4E454C2033330000000000434841DA
:100660004E4E454C20333400000000005649525491
:1006700055414C20310000000000005649525455AD
:10068000414C2032000000000000564952545541B0
:100690004C20330000000000005649525455414C94
:1006A00020340000000000005649525455414C20AF
:1006B000350000000000005649525455414C203688
:1006C0000000000000005649525455414C203700AC
:1006D00000000000005649525455414C203800009B
:1006E000000000005649525455414C20390000008A
:1006F0000000005649525455414C20313000000052
:1007000000005649525455414C2031310000000040
:10071000005649525455414C20313200000000002F
:100720005649525455414C203133000000000056C8
:1007300049525455414C20313400000000005649C4
:10074000525455414C2031350000000000564952AA
:100750005455414C20313600000000005649525497
:1007600055414C2031370000000000564952545585
:10077000414C203138000000000056495254554188
:100780004C20313900000000005649525455414C6C
:10079000203230000000000011241FBECFEFD0E156
:1007A000DEBFCDBF11E0A0E0B1E0E4EAFCEA00E08A
:1007B0000BBF02C007900D92AA37B107D9F71FE00F
:1007C000AAE7B1E001C01D92A935B107E1F70C9489
:1007D000842A0C940000282F2770992796958795D6
:1007E000969587959695879533272330310529F17E
:1007F000243031054CF421303105B9F02230310577
:10080000C4F4232B71F02CC025303105F1F02530D4
:100810003105BCF026303105E1F027303105E9F033
:100820001FC0A098A198A2981BC0A09AA198A298B6
:1008300017C0A098A19AA29813C0A09AA19AA298B2
:100840000FC0A098A198A29A0BC0A09AA198A29AB2
:1008500007C0A098A19AA29A03C0A09AA19AA29AAE
:10086000806280937C0080917A00806480937A001B
:1008700080917A0084FFFCCF80917A008061809320
:100880007A0020917800809179009927880F991F2C
:10089000880F991F2295269526952370820F911D0A
:1008A0000895282F2770992796958795969587956F
:1008B0009695879533272330310529F1243031056A
:1008C0004CF421303105B9F022303105C4F4232B2A
:1008D00071F02CC025303105F1F025303105BCF028
:1008E00026303105E1F027303105E9F01FC0A0982E
:1008F000A198A2981BC0A09AA198A29817C0A098EE
:10090000A19AA29813C0A09AA19AA2980FC0A098E9
:10091000A198A29A0BC0A09AA198A29A07C0A098E9
:10092000A19AA29A03C0A09AA19AA29A80628093E7
:100930007C0080917A00806480937A0080917A00B4
:1009400084FFFCCF80917A00806180937A0080914F
:1009500079009927089540E050E0FC010296259126
:1009600034916217730760F44B5F5F4FFC0102968E
:10097000259134916217730718F446395105A4F391
:10098000CA010895FC01809100018130B1F41092F8
:100990000001F0938301E0938201F0938101E093E1
:1009A0008001F0937F01E0937E01F0937D01E0935D
:1009B0007C01F0937B01E0937A016091800170915A
:1009C0008101709383016093820140917E01509177
:1009D0007F01509381014093800120917C013091EF
:1009E0007D0130937F0120937E0180917A01909167
:1009F0007B0190937D0180937C01F0937B01E093D8
:100A00007A01E80FF91FE20FF31FE40FF51FCF0182
:100A1000860F971F65E070E00E949955CB010895FD
:100A200080E10E94EB030E94C204BC018EE591E0CC
:100A30000E94AB049927089583E10E9451049FE42A
:100A4000899FC0011124880F892F881F990B9195C8
:100A5000A82F809101018130C1F4109201018A2FE9
:100A6000992790938D0180938C0190938B018093B3
:100A70008A019093890180938801909387018093E4
:100A800086019093850180938401E0918A01F09121
:100A90008B01F0938D01E0938C016091880170913E
:100AA000890170938B0160938A0140918601509176
:100AB00087015093890140938801209184013091EE
:100AC000850130938701209386018A2F992790937F
:100AD000850180938401820F931F840F951F860FD9
:100AE000971F8E0F9F1F65E070E00E949955862F1B
:100AF0009927089580E280937C0087E880937A00AC
:100B0000989A999A9A9AA098A198A298089590E094
:100B1000892F8295807F8093ED001092EE001092D5
:100B2000EF001092F0001092F1001092F20010927B
:100B3000F3001092F4001092F5001092F60010925B
:100B4000F70080E01092FA008F5F8830D8F39F5F43
:100B50009F30F0F208953091ED0090E020EC892F65
:100B60008295807F8093ED008091EF00822329F4AD
:100B70003093ED00892F992708959F5F9F3078F378
:100B80003093ED008FEF90E008958091EE0086FFA6
:100B900003C080E090E008958091EE0085FF03C0DF
:100BA00081E090E008958091EF00807C19F48FEF50
:100BB00090E0089582E090E00895BC0140E08091CB
:100BC000EF0099278F709070892B89F0FB01E40F5B
:100BD000F11D8091FA0080834F5F242F332780918D
:100BE000EF0099278F709070281739077CF30895CC
:100BF00081E09EE00E94D52967EA7EE080E00E94C5
:100C0000122A6FE57EE081E00E94122A69E17EE00F
:100C100082E00E94122A81E080938E018091010E71
:100C2000813061F48091020E9091030E6AE070E0D1
:100C30000E9499557093000E6093FF0D8091A80E4D
:100C4000813061F48091A90E9091AA0E6AE070E063
:100C50000E9499557093FC0D6093FB0D8091600E7E
:100C6000813061F48091610E9091620E6AE070E0D3
:100C70000E9499557093FE0D6093FD0D80911A0EA0
:100C8000813061F480911B0E90911C0E6AE070E03F
:100C90000E9499557093A60E6093A50E0895CF9368
:100CA000DF93CDB7DEB7CE55D0400FB6F894DEBF98
:100CB0000FBECDBF19828CE0888F84E690E09B83C5
:100CC0008A831D821C821E821F82188619861A86BC
:100CD0001B8689819E01245F3F4FF901E80FF11DBA
:100CE00010828F5F8C30C8F3CE0101960E94C52917
:100CF000A895198E1A8E84E690E09C8F8B8F1E8E9D
:100D00001D8E898D9E012F5F3F4FF901E80FF11D68
:100D1000168E8F5F8232C8F3CE0149960E94E52974
:100D2000A89581E0898F1A8E84E690E09C8F8B8F46
:100D30001E8E1D8E8A8D9E012F5F3F4FF901E80F99
:100D4000F11D168E8F5F8232C8F3CE0149960E9444
:100D5000E529A89582E0898F1A8E84E690E09C8F21
:100D60008B8F1E8E1D8E8A8D9E012F5F3F4FF90146
:100D7000E80FF11D168E8F5F8034C8F3CE014996BF
:100D80000E94E529C25ADF4F0FB6F894DEBF0FBEAE
:100D9000CDBFDF91CF91089599278832910509F44D
:100DA00040C08932910594F48532910559F186321B
:100DB000910534F483329105D9F08497F1F04FC056
:100DC0008632910521F1879739F149C08B3291051F
:100DD000B9F18C32910534F48932910539F18A9751
:100DE00051F13DC08C32910581F18D9799F137C059
:100DF00080EC0E940A379927089581EC0E940A37F7
:100E00009927089582EC0E940A379927089581ED69
:100E10000E940A379927089584EC0E940A3799277F
:100E2000089585EC0E940A379927089586EC0E9460
:100E30000A379927089587EC0E940A379927089561
:100E400083EC0E940A379927089582ED0E940A37A1
:100E50009927089583ED0E940A379927089580E025
:100E600090E00895FF920F931F93CF93DF93CDB738
:100E7000DEB765970FB6F894DEBF0FBECDBF809189
:100E8000FF0D9091000E009709F479C0019790939F
:100E9000000E8093FF0D892B09F071C08091020E26
:100EA0009091030E6AE070E00E9499557093000ED5
:100EB0006093FF0D8091040E9091050EAA27BB2729
:100EC00089839A83AB83BC8388E08D8380918E0174
:100ED0008E838091060E0E9428219695879596957F
:100EE00087958F838091070E0E942821969587957C
:100EF0009695879588878091080E0E94282196955F
:100F000087959695879589878091090E0E9428215B
:100F100096958795969587958A8780910A0E0E9467
:100F2000282196958795969587958B8780910B0EAE
:100F30000E94282196958795969587958C87209174
:100F40008E0181E09EE0FC01E20FF11D82850E948E
:100F5000282196958795969587958D8780918E0106
:100F6000982F9F5F90938E018091180E891718F427
:100F700081E080938E01CE0101960E943C358091E4
:100F8000FB0D9091FC0D009709F4BFC00197909361
:100F9000FC0D8093FB0D892B09F0B7C0CE010E9696
:100FA0000E9492208091A90E9091AA0E6AE070E0B2
:100FB0000E9499557093FC0D6093FB0D8091AB0ED0
:100FC0009091AC0EAA27BB2789839A83AB83BC83FD
:100FD00088E08D83FF2400E81F2D812F9927FC01D5
:100FE000E955F14F8681833230F40E944C208823EA
:100FF00031F0F02A04C00E94CC068111F02A069537
:101000001F5F183050F3FE82FF2400E81F2D812F50
:101010009927FC01E955F14F8685833230F40E940F
:101020004C20882331F0F02A04C00E94CC068111A4
:10103000F02A06951F5F183050F3FF82FF2400E866
:101040001F2D812F9927FC01E955F14F86898332A5
:1010500030F40E944C20882331F0F02A04C00E9412
:10106000CC068111F02A06951F5F183050F3F886E0
:10107000FF2400E81F2D812F9927FC01E955F14F2E
:10108000868D833230F40E944C20882331F0F02A80
:1010900004C00E94CC068111F02A06951F5F18300B
:1010A00050F3F986FF248091CD0E833248F40E94DC
:1010B0004C20882359F00F2EF0E8FF2EF02D06C0AB
:1010C0000E94CC06882311F080E8F82A8091CE0E89
:1010D000833238F40E944C20882349F080E4F82AB7
:1010E00006C00E94CC06882311F080E4F82AFA8614
:1010F0008E859F856AE070E00E9499556B871C86FB
:101100001D86CE0101960E943C358091FD0D909187
:10111000FE0D009709F4BBC001979093FE0D8093DC
:10112000FD0D892B09F0B3C08091610E9091620E84
:101130006AE070E00E9499557093FE0D6093FD0D7A
:101140008091630E9091640EAA27BB2789839A83AE
:10115000AB83BC8388E08D83FF2400E81F2D812FA3
:101160009927FC01E15AF14F8681833230F40E94C5
:101170007220882331F0F02A04C00E94CC0681112D
:10118000F02A06951F5F183050F3FE82FF2400E816
:101190001F2D812F9927FC01E15AF14F868583325B
:1011A00030F40E947220882331F0F02A04C00E949B
:1011B000CC068111F02A06951F5F183050F3FF828C
:1011C000FF2400E81F2D812F9927FC01E15AF14FE0
:1011D0008689833230F40E947220882331F0F02A0D
:1011E00004C00E94CC068111F02A06951F5F1830BA
:1011F00050F3F886FF2400E81F2D812F9927FC016A
:10120000E15AF14F868D833230F40E947220882398
:1012100031F0F02A04C00E94CC068111F02A069514
:101220001F5F183050F3F986FF248091850E8332BA
:1012300048F40E947220882359F00F2EF0E8FF2E08
:10124000F02D06C00E94CC06882311F080E8F82A11
:101250008091860E833238F40E947220882349F0F0
:1012600080E4F82A06C00E94CC06882311F080E4AE
:10127000F82AFA868E859F856AE070E00E9499556B
:101280006B871C861D86CE0101960E943C3580919D
:10129000A50E9091A60E009709F4F4C001979093C3
:1012A000A60E8093A50E892B09F0ECC080911B0E31
:1012B00090911C0E6AE070E00E9499557093A60E02
:1012C0006093A50E80911D0E90911E0EAA27BB273C
:1012D00089839A83AB83BC8388E08D83FF2400E8F5
:1012E0001F2D812F9927FC01E75EF14F8681833204
:1012F00030F40E944C20882331F0F02A04C00E9470
:10130000CC068111F02A06951F5F183050F3FE823B
:10131000FF2400E81F2D812F9927FC01E75EF14F84
:101320008685833230F40E944C20882331F0F02AE5
:1013300004C00E94CC068111F02A06951F5F183068
:1013400050F3FF82FF2400E81F2D812F9927FC0115
:10135000E75EF14F8689833230F40E944C20882367
:1013600031F0F02A04C00E94CC068111F02A0695C3
:101370001F5F183050F3F886FF2400E81F2D812FDF
:101380009927FC01E75EF14F868D833230F40E948D
:101390004C20882331F0F02A04C00E94CC06811131
:1013A000F02A06951F5F183050F3F986FF2400E8F5
:1013B0001F2D812F9927FC01E75EF14F86A1833213
:1013C00030F40E947220882331F0F02A04C00E9479
:1013D000CC068111F02A06951F5F183050F3FA866B
:1013E000FF2400E81F2D812F9927FC01E75EF14FB4
:1013F00086A5833230F40E947220882331F0F02ACF
:1014000004C00E94CC068111F02A06951F5F183097
:1014100050F3FB86FF2400E81F2D812F9927FC0144
:10142000E75EF14F86A9833230F40E947220882350
:1014300031F0F02A04C00E94CC068111F02A0695F2
:101440001F5F183050F3FC86FF2400E81F2D812F0A
:101450009927FC01E95AF14F8081833230F40E94D0
:101460007220882331F0F02A04C00E94CC0681113A
:10147000F02A06951F5F183050F3FD86CE010196C5
:101480000E943C3565960FB6F894DEBF0FBECDBF07
:10149000DF91CF911F910F91FF9008958F929F92AE
:1014A000BF92CF92DF92EF92FF920F931F93CF9351
:1014B000DF93CDB7DEB7EC970FB6F894DEBF0FBE63
:1014C000CDBFBB240F2EF3E18F2E9924F02DBE014A
:1014D0006F5F7F4F8B2D0E94FB278B2D9927889D57
:1014E0009001899D300D989D300D1124F901E1572F
:1014F000FE4F9981492F41708081887F9670842B9F
:10150000892B80830F2EFFE8CF2EF1E0DF2EF02D08
:10151000C20ED31E8A819B81F601928381838C81C6
:101520009D81948383832E813F81368325838885A3
:101530009985908787839A8591878B8582878C850B
:1015400083878D8584878E8585878F8586878F8D18
:10155000878788A1808B89A1818B8AA1828B933018
:1015600090F5C901AA2797FDA095BA2FBC01CD011E
:101570000E94B152DC01CB0128A539A54AA55BA583
:10158000BC01CD010E94CB517B018C018CA5992718
:1015900087FD9095A92FB92FBC01CD010E94B152B2
:1015A000DC01CB019C01AD01C801B7010E9496513D
:1015B000DC01CB01BC01CD010E941750DC01CB0145
:1015C000F601968385838B2D9927889D9001899DAF
:1015D000300D989D300D11240F2EFFE8CF2EF1E035
:1015E000DF2EF02DC20ED31EF6018285833098F5D2
:1015F00088859985AA2797FDA095BA2FBC01CD01B2
:101600000E94B152DC01CB0128A539A54AA55BA5F2
:10161000BC01CD010E94CB517B018C018CA5992787
:1016200087FD9095A92FB92FBC01CD010E94B15221
:10163000DC01CB019C01AD01C801B7010E949651AC
:10164000DC01CB01BC01CD010E941750DC01CB01B4
:10165000F601908787832B2D3327289DC001299D74
:10166000900D389D900D1124FC01E157FE4F8081B3
:1016700086958370813029F4F901E151FC4F808314
:1016800006C08B2D9927FC01E151FC4F10828B2D58
:101690009927FC01E25EFB4F1082B394FFE1FB153A
:1016A00008F015CFFE01BD96A0E0B9E080E190E022
:1016B00021E08030920719F40E943C5603C0182E96
:1016C0000E943C568DA580931C048EA580931D041A
:1016D0001092100410920F04EC960FB6F894DEBF2F
:1016E0000FBECDBFDF91CF911F910F91FF90EF9073
:1016F000DF90CF90BF909F908F9008951F93CF93CE
:10170000DF93CDB7DEB7EC970FB6F894DEBF0FBE10
:10171000CDBF10E0A8958981887F89831B821A82BA
:101720001D821C821F821E82198618861A861B86BD
:101730001C8681E08D871E868F871F8E18A219A2B6
:101740001AA280E090E0A0E8BFE388A799A7AAA723
:10175000BBA71CA685E0FE01B39611928A95E9F716
:101760008FE0FE017096DF01282F1D922A95E9F780
:10177000189FC001112482569E4FBC01CF010E94C8
:101780003C55BE016F5F7F4F812F0E94C3271F5FB3
:10179000103208F4BFCFFE01BD9680E1DF011D923B
:1017A0008A95E9F7A0E0B9E080E190E021E080309F
:1017B000920719F40E944D5603C0182E0E944D56F0
:1017C000EC960FB6F894DEBF0FBECDBFDF91CF9180
:1017D0001F91089580930F0408950F93CF93DF9383
:1017E000CDB7DEB721970FB6F894DEBF0FBECDBFE1
:1017F00089838150803270F000E021E0AE014F5FBC
:101800005F4F63EF70E082E091E00E94C62380E0CA
:1018100090E007C089819927FC01E251FC4F80814B
:10182000992721960FB6F894DEBF0FBECDBFDF918A
:10183000CF910F9108951F93CF93DF9380911C0454
:10184000882381F080911D040E940A37882351F477
:10185000582F8FEE93E0FC01E50FF11D10825F5FC2
:101860005032C8F350E06EE174E0A3E1B0E0CFEE97
:10187000D3E011E0252F3327F901E60FF71F808110
:10188000882309F1482F415040834423E1F42A9FE3
:10189000C0012B9F900D3A9F900D1124FC01E15740
:1018A000FE4F80818695837099278130910539F0AC
:1018B000029749F0F901EC0FFD1F408304C0FE01BF
:1018C000E50FF11D10835F5F5032A0F2DF91CF91E1
:1018D0001F91089580910F04882399F0809110043E
:1018E000882379F080E194E0AC014C5F5F4F609118
:1018F000130480911104909112040E940B421092E3
:1019000010040895AF92BF92CF92DF92EF92FF92B0
:101910000F931F93CF93DF938C01EE24FF24BB24FE
:1019200080911C04882339F080911D040E940A379D
:10193000882309F400C260E070910F040F2EFFEEBF
:10194000CF2EF3E0DF2EF02DAA24A39483E1689F2D
:10195000C0011124EC01C157DE4F89819A81AA2769
:1019600097FDA095BA2FF8012081318142815381E2
:1019700082179307A407B50759F08B819C81AA278A
:1019800097FDA095BA2F82179307A407B507A9F46E
:10199000462F5527FA01E25EFB4F8FE08083872FA9
:1019A000733048F099279C012F733070CA01039659
:1019B0002817390711F4BB24B3948F85882349F085
:1019C0008889F801E80FF11D99898581981709F038
:1019D0005FC129813A812115310509F459C1442794
:1019E00037FD4095542FF80180819181A281B38108
:1019F000281739074A075B0709F09CC091E08B85DF
:101A0000882379F0E80FF11D8481E82EFF24FE2C55
:101A1000EE248C85F801E80FF11D8481E80EF11C9D
:101A200014C08C85882381F0F801E80FF11D8481B2
:101A3000E82EFF248A89813041F4EE2034F420E03E
:101A40003FEFE22AF32A01C090E0992309F472C023
:101A50008985992782309105B9F1833091052CF45D
:101A6000009779F00197C1F065C08430910509F4C1
:101A70004DC0843091050CF43EC0059709F451C067
:101A800059C08D819E818E159F0509F053C0F601C6
:101A9000E60FF11DA0824EC02A89213059F48D81B4
:101AA0009E818E159F050CF045C0F601E60FF11DD5
:101AB000208340C08D819E818E159F05D8F5F6014B
:101AC000E60FF11DA08236C02A89213051F48D81A4
:101AD0009E81E816F90674F5F601E60FF11D2083E4
:101AE00029C08D819E81E816F90620F5F601E60FE2
:101AF000F11DA0821FC08D819E818E219F21892B87
:101B0000C9F0F601E60FF11DA08214C08D819E81FF
:101B10008E219F21892B71F4F601E60FF11DA08221
:101B200009C08D819E818E159F0521F0F601E60F7B
:101B3000F11DA0828B819C819C01442737FD40953B
:101B4000542FF80180819181A281B3812817390730
:101B50004A075B0709F09CC091E08D85882379F0E6
:101B6000E80FF11D8481E82EFF24FE2CEE248E85E3
:101B7000F801E80FF11D8481E80EF11C14C08E8578
:101B8000882381F0F801E80FF11D8481E82EFF24FD
:101B90008A89813041F4EE2034F420E03FEFE22ADC
:101BA000F32A01C090E0992309F472C08A8599272D
:101BB00082309105B9F1833091052CF4009779F0CA
:101BC0000197C1F065C08430910509F44DC084309F
:101BD00091050CF43EC0059709F451C059C08F819E
:101BE00098858E159F0509F053C0F601E60FF11D8B
:101BF00010824EC08A89813059F48F8198858E1564
:101C00009F050CF045C0F601E60FF11D108240C0A3
:101C10008F8198858E159F05D8F5F601E60FF11D89
:101C2000108236C08A89813051F48F819885E816F8
:101C3000F90674F5F601E60FF11D108229C08F81B7
:101C40009885E816F90620F5F601E60FF11D1082D9
:101C50001FC08F8198858E219F21892BC9F0F601A5
:101C6000E60FF11D108214C08F8198858E219F216F
:101C7000892B71F4F601E60FF11D108209C08F81E6
:101C800098858E159F0521F0F601E60FF11D108253
:101C90006F5F603208F45ACE80910F04882309F4F4
:101CA0004AC0BB2019F4823009F045C0809110046D
:101CB000823009F440C080911104909112049C017B
:101CC00044275527F80180819181A281B38128178B
:101CD00039074A075B0799F4909113048481981798
:101CE00071F4892F992798012B5F3F4FAC01B901FF
:101CF00080E194E004960E944355892BC9F082E06C
:101D000080931004F8012481209313048081918131
:101D10009093120480931104822F992798012B5FCE
:101D20003F4FAC01B90184E194E00E94505503C0DB
:101D300081E080931004DF91CF911F910F91FF906C
:101D4000EF90DF90CF90BF90AF90089582E08093A6
:101D5000E20084E08093E30083E18093E4000E944A
:101D600087058091D80082608093D8000895CF9332
:101D7000DF93EC018981833089F48985882309F414
:101D800003C188818295807F8093ED008091EF0070
:101D90008F738093EF0018821986F6C00E94AB05FE
:101DA000982F81E089879F3F09F4EBC09883892FA2
:101DB0008295807F8093ED001092EE001092EF00EC
:101DC0001092F7001092F6001092F5001092F400B5
:101DD0001092F000898199278130910509F46BC038
:101DE000823091051CF4892B29F0C9C0029709F4AF
:101DF000BBC0C5C08A8581FF30C08D81982F990FE7
:101E0000990F990F8C81829586958770890F8093A1
:101E1000F3008C81982F990F990F990F8B818295E0
:101E200086958770890F8093F2008B81982F990F88
:101E3000990F990F8A81829586958770890F809373
:101E4000F1008A81880F880F880F8093F0008091BD
:101E5000EF0080618093EF0012C08B81982F9295E4
:101E6000990F907E8A81869586958695890F8093B5
:101E7000F3008A818295880F807E8093F20020E0B3
:101E80008E81181660F48F819885FC01E20FF11D98
:101E900080818093FA002F5F8E812817A0F39091A4
:101EA000EF008E81892B8093EF008091EF0080649A
:101EB0008093EF0069C08A8581FF35C08D81982F9E
:101EC000990F990F990F8C81829586958770890F4C
:101ED0008093F3008C81982F990F990F990F8B8124
:101EE000829586958770890F8093F2008B81982F59
:101EF000990F990F990F8A81829586958770890F1E
:101F00008093F1008A81880F880F880F8093F000FA
:101F10008091EF0080618093EF008091F0008460F9
:101F20008093F00015C08B81982F9295990F907E29
:101F30008A81869586958695890F8093F3008A819C
:101F40008295880F807E8093F20084E08093F00079
:101F50009091EF008E81892B8093EF008091EF00AC
:101F600080648093EF0010C08091EF008F738093A6
:101F7000EF008091EF0080688093EF0005C0198624
:101F800003C08FEF90E002C080E090E0DF91CF913E
:101F90000895CF93DF93EC018985882319F482E0BB
:101FA00090E082C088818295807F8093ED000E94BE
:101FB000C505813009F06CC019868091EF008F70E3
:101FC0008E838F8198850E94DD058091F00099278E
:101FD000847090709595879595958795982F9170B9
:101FE0008A85282F2E7F292B2A878091EF0084FF56
:101FF00031C0822F82608A878091F3008695869512
:1020000086958D838091F200982F9695969596955A
:102010008091F3008295880F807E890F8C83809158
:10202000F100982F9695969596958091F20082955D
:10203000880F807E890F8B838091F000982F969572
:10204000969596958091F1008295880F807E890FF4
:102050008A8316C08A858D7F8A878091F300829556
:10206000869587708B838091F200982F9295969534
:1020700097708091F300880F880F880F890F8A83EB
:102080008091EF008F738093EF0080E090E00CC0B0
:10209000882349F489878091EF008F738093EF0044
:1020A00080E090E001C09927DF91CF91089586EB01
:1020B00099E00E941E220E94FB1008951F93CF9367
:1020C000DF930E942A180E94BD170E94661910E033
:1020D00087E2189FC0011124EC01CB5BDB4F8C8998
:1020E0009D89009719F001979D8B8C8B8D859E851E
:1020F000009761F001979E878D8799859F3F31F00A
:1021000085E0989FC00111249B878A872A853B859B
:102110002115310561F089858F3F49F0C90101978B
:102120009B878A87892B19F48F8580628F878B8D97
:102130009C8D009779F001979C8F8B8F892B51F4A0
:102140008F8586FD04C0812F8F5F0E94A4268F8516
:1021500080648F878F81882311F081508F831F5F68
:10216000123208F4B5CFDF91CF911F91089590916D
:10217000AD098091BD099817E0F420E04DEB59E0DE
:1021800067E270E0FA01E20FF11D8281823268F4A9
:102190009927869FF001879FF00D969FF00D1124DF
:1021A000E75BFB4F8081816080832F5F2C3050F391
:1021B00008959091AD098091BE098917D8F420E067
:1021C0004DEB59E067E270E0FA01E20FF11D828108
:1021D000823268F49927869FF001879FF00D969FC1
:1021E000F00D1124E75BFB4F80818E7F80832F5F92
:1021F0002C3050F30895CF92DF92EF92FF920F931D
:102200001F93CF93DF9380913F04882309F0FDC093
:10221000F82E0F2EFAE0EF2EF02D8DE0F89EC00183
:102220001124EC01CC51D64F00E08A818F3F11F48C
:1022300001E01DC09A81892F805C843128F4892FA8
:102240000E940A37082F13C09A81892F815080324B
:1022500028F4892F0E94ED0B082F09C09A81892F3D
:102260008152843120F4892F0E94E047082F898110
:10227000992781309105C9F1823091051CF4892B91
:1022800029F0BEC0029709F4B8C0BAC0013009F005
:10229000B7C08F818E9DC00111249C838B8388855C
:1022A0008E9DC00111249E838D83888184608883E4
:1022B00010E027E230E0FE01E10FF11D81858F3F44
:1022C00071F09927829FA001839F500D929F500D1E
:1022D0001124FA01E75BFB4F8081846080831F5FDC
:1022E000143048F381E089838BC08B819C810097F7
:1022F00009F486C001979C838B83892B49F58F81D4
:102300008E9DC00111249C838B83888182FF10C025
:102310008B7F888310E0FE01E10FF11D81858F3FE7
:1023200019F060E00E940E121F5F1430A0F310C07D
:1023300088818460888310E0FE01E10FF11D8185B2
:102340008F3F19F061E00E940E121F5F1430A0F35E
:102350008881282F227081FD28C08D819E81009761
:1023600009F44EC001979E838D83892B09F048C0E4
:1023700082E08983122F27E230E0FE01E10FF11D98
:1023800081858F3F71F09927829FA001839F500D17
:10239000929F500D1124FA01E75BFB4F80818B7FE8
:1023A00080831F5F143048F32BC0002349F5102FA2
:1023B0000F2EF7E2CF2EDD24F02DFE01E10FF11DEF
:1023C00021852F3F99F0822F99278C9DA0018D9D0B
:1023D000500D9C9D500D1124FA01E75BFB4F80814D
:1023E0008B7F808361E0822F0E940E121C821B82F1
:1023F0001F5F143010F3198203C0002309F409830E
:10240000F39454E05F1508F008CFDF91CF911F914E
:102410000F91FF90EF90DF90CF900895DF92EF92B1
:10242000FF920F931F93CF93DF93CDB7DEB7219722
:102430000FB6F894DEBF0FBECDBF8983162FDD2403
:10244000833260F00D2D21E0AE014F5F5F4F67ECEE
:1024500071E082E191E00E94C6234EC0998187E23B
:10246000989F7001112485E494E0E80EF91EF701AD
:10247000868D9927807F9070803A910529F40F2EE0
:10248000F1E4DF2EF02D18C0F701868D9927807FAB
:102490009070803B910529F40F2EF2E4DF2EF02D91
:1024A0000BC000E021E0AE014F5F5F4F63ED71E0D4
:1024B00082E191E00E94C623112379F483E0F701C1
:1024C000878380EF818387858F7B8787868D42A175
:1024D0006D2D8F700E94902F0FC0113069F4F7019D
:1024E00017828FE08183878586798787868D42A1D1
:1024F0006D2D8F700E94DB2F21960FB6F894DEBFF2
:102500000FBECDBFDF91CF911F910F91FF90EF9044
:10251000DF90089520E04BEC59E067E270E08170B5
:10252000382F330FFA01E20FF11D8181823270F4EE
:102530009927869FF001879FF00D969FF00D11243B
:10254000E75BFB4F80818D7F832B80832F5F203162
:1025500048F3089580914104909142040895809138
:10256000400499270895EF92FF921F93CF93DF9332
:102570007A018093BD096093BE0910E0C12FDD2769
:10258000F701EC0FFD1F80810E94B91E823220F4FA
:10259000FE01E354F64F82831F5F1C3078F3DF9116
:1025A000CF911F91FF90EF9008959F92AF92BF92AD
:1025B000CF92DF92EF92FF920F931F93CF93DF930F
:1025C000CDB7DEB722970FB6F894DEBF0FBECDBFF2
:1025D00099240E94AC200E949B210E94C62186EB78
:1025E00099E00E9413221092AB091092AA099092CE
:1025F000AC099092AE099092AF099092B009909276
:10260000B10982E1E3E7F9E011928A95E9F745E83B
:1026100059E028EB31E0892D9927880F991FFC019B
:10262000E40FF51F31832083939461E1691598F7D6
:10263000992444EE59E02DE030E0892D9927829FBE
:10264000F001839FF00D929FF00D1124CF01E40F54
:10265000F51F11821482138216821582FC01EC513F
:10266000F64F8081846080839394F4E0F91528F715
:102670000E94532A803221F487E68093110103C01F
:102680008EE6809311010F2EF5E4AF2EF4E0BF2EFD
:10269000F02D21E02093450448EC50E0509358047D
:1026A0004093570432EA3093630462EB609364040E
:1026B000109267049FEF909365043093660415E0D1
:1026C0001093680483E0809369040F2EF7E2CF2E05
:1026D000DD24F02DCA0CDB1C20936C04F50152AFF5
:1026E00041AFF601368F678F22A390A30F2EF7EA32
:1026F000FF2EF02DF1A213A38FE084A3F501E25B7E
:10270000FF4F20939304538B428B0F2EF3EAEF2E4F
:10271000F02DE68E83EB878F22A390A391A393A342
:1027200089E084A3F501EB58FF4F2093BA04538B43
:10273000428BF68E0F2EF7EBCF2EF02DC78E22A3F5
:1027400090A391A393A38BE084A3F501E456FF4FDC
:102750002093E104538B428B0F2EF1EADF2EF02DF4
:10276000D68E81EB878F22A390A391A393A38EE0B3
:1027700084A3F501ED53FF4F20930805538B428B43
:1027800035EA368F05EB078F22A390A391A393A37D
:102790008DE084A30F2EF6E09F2EF02DF501E6517B
:1027A000FF4F20932F05538B428B60EA668F70EBAF
:1027B000778F12A290A331A313A394A2F501EF5E29
:1027C000FE4F20935605538B428B368F078F12A2F4
:1027D00090A391A393A384E084A3F501E85CFE4F4A
:1027E00020937D05538B428B668F778F22A390A316
:1027F00061A313A38AE084A3F501E15AFE4F20935D
:10280000A405538B428B768F34EB378F12A390A3A2
:1028100091A393A382E184A3F501EA57FE4F20938D
:10282000CB05538B428B64EA668F378F22A390A32C
:10283000E1A213A388E084A3F501E355FE4F2093A2
:10284000F205538B428B36EA368F86EB878F12A2C6
:1028500090A361A313A324A30F2EFCE09F2EF02DC1
:10286000F501EC52FE4F20931906538B428B368FA5
:10287000878F22A390A3D1A213A394A2F501E550C0
:10288000FE4F20934006538B428BF68EC78E12A2CA
:1028900090A391A393A3CC246894C1F8C4A29501FA
:1028A000F501EE5DFD4F71E070936706538B428B2F
:1028B000BD2CD68E0F2EF1EBEF2EF02DE78E12A24F
:1028C00090A391A393A387E084A3F901E75BFD4F55
:1028D00070938E06538B428BE68EF02E078F612FFE
:1028E00012A390A391A393A381E184A3F901E059DA
:1028F000FD4F7093B506538B428B14EA168F0F2E43
:10290000F4EBDF2EF02DD78E12A290A386EA81A3DE
:1029100063A364A3F901E956FD4F7093DC06538B62
:10292000428B0F2EF3EAAF2EF02DA68E03EB078F0E
:1029300012A290A391A393A314A2F901E254FD4F14
:1029400070E4709303074FEF5FEF538B428BA7EA5E
:10295000A68FD78E63E062A380A391A393A394A3D1
:10296000F901EB51FD4F70932A07538B428B868FF1
:10297000F78E62A380A391A393A394A3F901E45FCC
:10298000FC4F70935107538B428B0F2EF5EA9F2E0D
:10299000F02D968E86EB878F62A3A0A391A393A3BD
:1029A00094A3F901ED5CFC4F70937807538B428B35
:1029B000168F87EB878F62A3A0A391A393A394A301
:1029C000F901E65AFC4F70939F07538B428B0F2EF1
:1029D000F0EADF2EF02DD68E078F62A390A291A38E
:1029E00093A394A3F901EF57FC4F7093C607538B41
:1029F000428BB68EA2EBA78F62A390A291A393A362
:102A000094A3F901E855FC4F7093ED07538B428B6B
:102A100082EA868FE78E62A310A391A393A394A367
:102A2000F901E153FC4F70931408538B428BA68E2F
:102A300080EB878F62A310A391A393A394A3F901C2
:102A4000EA50FC4F70933B08538B428BD68E078F16
:102A5000C2A2F0A291A393A394A3F901E35EFB4F5A
:102A600070936208538B428BB68EA78FC2A2F0A2DE
:102A700091A393A3F901E35EFB4F94A3B901F9017C
:102A8000EC5BFB4FA0E4A0938908538B428B82EA56
:102A9000868FE78EC2A224EB20A391A393A394A3D5
:102AA000FB01E559FB4FA093B008538B428BA68ED8
:102AB00080EB878FC2A220A391A393A394A3FB01D1
:102AC000EE56FB4FA093D708538B428B87EA868F35
:102AD000278FC2A226EB20A391A393A394A3FB016B
:102AE000E754FB4FA093FE08538B428B86EA868FF8
:102AF000F78EC2A220A391A393A394A3FB01E0525B
:102B0000FB4FA0932509538B428B968E278FC2A231
:102B100027EB20A391A393A394A3FB01E95FFA4FB2
:102B2000A0934C09538B428B168F278FC2A220A3F0
:102B300091A393A394A3992447E250E02FE0B92FE7
:102B400001E21EE130E1892D9927849FF001859FE4
:102B5000F00D949FF00D1124CF017F01E60EF71EBA
:102B6000F701158A148A168A875B9B4F9A8389839B
:102B7000FC0180818C7F8083F7011786178A21836F
:102B800016A215A216861586148613861286B1879C
:102B9000E981FA8180818B7F8083F701108E178213
:102BA0000087168335832283128E118E148E138E26
:102BB000158E9394F1E2F91530F622960FB6F8943B
:102BC000DEBF0FBECDBFDF91CF911F910F91FF9060
:102BD000EF90DF90CF90BF90AF909F900895E3E784
:102BE000F9E082E1DF011D928A95E9F7CF010E94A9
:102BF000852920E065E879E048EB51E0822F9927AC
:102C0000880F991FFC01E60FF71F518340832F5F48
:102C10002231A0F385E899E00E94A5290895AF929A
:102C2000BF92CF92DF92EF92FF920F931F93CF93B9
:102C3000DF93CDB7DEB7C456D0400FB6F894DEBFF1
:102C40000FBECDBFDD240F2EF5E1EF2EFF24F02DBA
:102C5000EC0EFD1E2D2D332787E290E0289FA0016A
:102C6000299F500D389F500D1124FA01EB5BFB4F4B
:102C700082899389892F99278D8B82898E8B868172
:102C80008F8B1A8E198E1B8E8581888F80858C8FF5
:102C90008FE0D89EC001112482599B4FBC01CE0108
:102CA0004D960E943C551CA68FEF8DA71D2D1F5FD2
:102CB000612FC7010E94A328A895D12E51E2511778
:102CC00048F684E68EA788E78FA74CE050E06FEFC8
:102CD00070E0CE01C0960E945D55CE018E960E9496
:102CE000E32681EC8CAF40E150E06FEF70E0CE0165
:102CF000CD960E945D55CE01CC960E941127A895D5
:102D0000DD240F2EF4E1CF2EF02D7E010894E11C7E
:102D1000F11C0FE0D701EC2D1D92EA95E9F7D09E4A
:102D2000C001112487539C4FBC01C7010E943C5530
:102D3000188A1D2D1F5FB701812F0E943A29D12EBD
:102D4000FAE0F11738F7A895DD240F2EF6E5AF2E3F
:102D5000BB24F02DAC0EBD1E0F2EFFE0EF2EF02D8C
:102D60008E01035B1F4FFF24FA94D501EE2D1D92B7
:102D7000EA95E9F7DE9CC001112482589C4FBC0102
:102D8000C80109960E943C55D8011C92F801118295
:102D9000128281E083838AE084838081F801E80FD6
:102DA000F11DF5828F5F8430C8F3BE01635B7F4FF6
:102DB0008D2D0E945127D394F4E0FD15B0F6ECED73
:102DC000F9E088E0DF011D928A95E9F7CF010E94C2
:102DD00031270E948E21CC59DF4F0FB6F894DEBF09
:102DE0000FBECDBFDF91CF911F910F91FF90EF905C
:102DF000DF90CF90BF90AF9008950F931F93CF9324
:102E0000DF93CDB7DEB7E1970FB6F894DEBF0FBE04
:102E1000CDBF00E0102F1F5F612FCE0101960E94F1
:102E2000E828202F332787E290E0289FA001299FE0
:102E3000500D389F500D1124FA01EB5BFB4F898137
:102E40009927982F88272A81820F911D938B828B37
:102E50008B818683888580878C818583888D848714
:102E6000898D81878D819E81928F818F8F81858FC2
:102E7000012F123278F28DEB99E00E9401278BEC42
:102E800099E00E94212783E799E00E94952985E82F
:102E900099E00E94B5298CED99E00E9441270E949B
:102EA0008E2100E0BE01665E7F4F802F0E948A2740
:102EB000202F33278DE090E0289FA001299F500DFF
:102EC000389F500D11249A01FA01EC51F64F8A8D6A
:102ED000582F51708081482F4C7F8B8D8170982F97
:102EE000990F842F852B892B8083F901EC51F64FA4
:102EF0008C8D82838D8D87838E8D8087F901E35140
:102F0000F64F8F8D98A1A9A1BAA180839183A28346
:102F1000B3830F5F053030F2E1960FB6F894DEBF51
:102F20000FBECDBFDF91CF911F910F910895CF9329
:102F3000DF93EC01862F0E94B91E8332D8F4282F2C
:102F4000332787E290E0289FA001299F500D389FEA
:102F5000500D1124FA01EB5BFB4F8F898487888128
:102F60009927982F88272981820F911D938B828B17
:102F70008A818683DF91CF9108959091CB09892F23
:102F80008150803268F4892F0E94ED0B882321F054
:102F900081E00E948A12089580E00E948A120895BA
:102FA0009091CB09892F8152843168F4892F0E9436
:102FB000E047882321F081E00E948A12089580E092
:102FC0000E948A1208958091CB090E940A378E3F91
:102FD00041F0813019F40E948A12089580E00E9425
:102FE0008A120895FC0184818860848380EF828343
:102FF000878586798787178A168A848525E0829F48
:10300000C001112496878587892B41F481858F3FE4
:1030100029F0829FC00111249387828783E08783F0
:1030200008951F93CF93C0E017E2C19FC001112400
:10303000FC01EB5BFB4F8785992783FD02C080FF76
:1030400003C0CF010E94F217CF5FC23270F3CF915D
:103050001F910895FF920F931F93CF93DF9310E07A
:103060000F2EFFE0FF2EF02D82E00E948C3787E2CA
:10307000189FC0011124EC01CB5BDB4F88858823AE
:1030800061F48981803F09F0CCC08C8188608C8399
:103090008F85867B8F87FA82C4C02885822F8150D6
:1030A0008032D0F58F85992783FD24C080FD22C012
:1030B000822F0E94ED0B882341F089818F3009F027
:1030C000B0C0CE010E94F217ACC08981803F09F0E8
:1030D000A8C089858F3F09F4A4C08A859B85892B68
:1030E00009F09FC08C8188608C838F85867B8F8759
:1030F000FA8297C088850E94ED0B882309F091C061
:103100008981803F09F08DC08C8188608C838F8598
:10311000867B8F87FA8285C02885822F81528431F1
:10312000D0F58F85992783FD24C080FD22C0822F92
:103130000E94E047882341F089818F3009F071C0F7
:10314000CE010E94F2176DC08981803F09F069C0ED
:1031500089858F3F09F465C08A859B85892B09F095
:1031600060C08C8188608C838F85867B8F87FA8294
:1031700058C088850E94E047882309F052C08981A1
:10318000803F09F04EC08C8188608C838F85867B60
:103190008F87FA8246C000E088850E940A37982F00
:1031A0008E3FA9F08885803C21F49130A1F4092F4D
:1031B00012C08D81813021F4913011F4092F0BC0A0
:1031C0008D81803141F4992331F401E004C0888578
:1031D0008F3F09F401E0002369F089818F3009F500
:1031E0008F85992783FD1DC080FD1BC0CE010E94E5
:1031F000F21717C08981803F31F08F85992783FDB1
:1032000002C080FF0EC089858F3F59F08A859B855B
:10321000892B39F48C8188608C838F85867B8F879E
:10322000FA821F5F123208F41FCFDF91CF911F91F6
:103230000F91FF90089560933F04623019F48FEF6F
:103240008093A9090895CF93DF93EC018881815081
:10325000823218F080E090E036C088810E94B91E6A
:10326000282F898199278F30910521F0803F910582
:10327000A1F027C0332787E290E0289FA001299F73
:10328000500D389F500D1124FA01EB5BFB4F8FE07E
:1032900081838785867F878714C0332787E290E004
:1032A000289FA001299F500D389F500D1124FA012D
:1032B000EB5BFB4F80EF81838785867F8787178A4B
:1032C000168A81E090E0DF91CF9108958F929F92CE
:1032D000AF92BF92CF92DF92EF92FF920F931F9324
:1032E000CF93DF93CDB7DEB721970FB6F894DEBF4B
:1032F0000FBECDBFBB24B9828B2CAB2C9B2C109264
:10330000AB091092AA09B092AE09B092B009B0927E
:10331000AF090E941C058093AD0980913F0488236A
:1033200009F073C2B9828B2D823208F0EDC482E0BD
:103330000E948C378824998187E2989FC0011124CC
:103340000F2EF5E4CF2EF4E0DF2EF02DC80ED91E9F
:10335000F601868D9927807F9070803A910529F437
:103360000F2EF1E4AF2EF02D18C0F601868D9927AF
:10337000807F9070803B910529F40F2EF2E4AF2EF0
:10338000F02D0BC000E021E0AE014F5F5F4F68E21F
:1033900076E082E191E00E94C623F601118A108A4C
:1033A000248122FDBCC0808199278130910509F4D8
:1033B0005DC08034910509F0BFC0818199278F30AD
:1033C0009105B1F1803F910509F0B6C0822F83705D
:1033D00019F4878585FF09C0F601868D42A16A2D03
:1033E0008F700E94DB2F882410C0F601858596859A
:1033F000892B59F4878580FD08C0868D42A16A2DEE
:103400008F700E94902F88248394F601848183FF1B
:1034100093C0877F848382818F3009F08DC0818340
:10342000868D42A16A2D8F700E94DB2F882484C074
:10343000F601248123FF80C0822F877F84838281CD
:10344000803F09F079C0818385859685892B09F0B5
:1034500073C0822F837009F06FC0868D42A16A2DE0
:103460008F700E94902F8824839466C0F60181811A
:1034700099278F309105C1F1803F910509F05CC01B
:103480008481837019F4878585FF09C0F601868DD4
:1034900042A16A2D8F700E94DB2F882413C0F60191
:1034A00085859685892B71F48785992780FD0AC0CB
:1034B00083FD08C0868D42A16A2D8F700E94902FD7
:1034C00088248394F601848183FF36C0877F8483B8
:1034D00082818F3089F58183868D42A16A2D8F701C
:1034E0000E94DB2F882428C0F601248123FF24C0FA
:1034F000822F877F84838281803FF1F48183858559
:103500009685892BC9F4822F8370B1F4868D42A1F0
:103510006A2D8F700E94902F882483940DC0F6012D
:10352000818199278F30910531F0803F910521F4F9
:103530008824839401C08824F6018181803F09F0AA
:1035400058C084A18F3F09F454C00E94EB037C0152
:1035500000271127F601F6A2E5A289819927FC012F
:10356000ED58F64F80819927AA27BB278E159F0516
:10357000A007B10724F0EE24FF2487010AC0898147
:103580009927FC01ED58F64F8081E81AF1080109EE
:103590001109F3E0EF16F10401051105CCF0898162
:1035A0009927880F991FFC01EB57F64F8081918175
:1035B0009C0144275527C801B7010E946E5520EE93
:1035C00031E040E050E00E94E25579018A0103C0F9
:1035D000EE24FF248701F601F18AE08A8091AA098E
:1035E0009091AB098E0D9F1D9093AB098093AA0912
:1035F00003C0F601118A108A882039F4F601838D00
:10360000948D892B11F0148E138EF60187859927DE
:10361000AC014870507083FD66C020893189828971
:10362000938982179307A0F5838D948D892B11F0D0
:10363000548F438FF60186898130F9F48489958906
:10364000892B09F050C08785886087878091AE09F3
:103650008F5F8093AE098081813039F4868D42A1DD
:103660006A2D8F700E94DB2F88248981F601608982
:1036700071898F5F0E94392636C081E0F601868B02
:10368000968185E0989FC0011124958B848B2BC077
:10369000F601168A218D328D2115310521F1882000
:1036A000A1F0808991898217930778F4838D948D96
:1036B000892BC9F4878586FD16C0958D85E0989F76
:1036C000C0011124948F838F0EC0F601838D948DD9
:1036D000892B49F020893189818D928D821793073A
:1036E00010F4148E138EF601878D9927807F9070C9
:1036F000803A910529F40F2EF1E49F2EF02D18C089
:10370000F601878D9927807F9070803B910529F481
:103710000F2EF2E49F2EF02D0BC000E021E0AE0151
:103720004F5F5F4F6EE377E082E191E00E94C62336
:10373000F601878D42A1692D8F700E945E30282F7F
:10374000F6018181803F09F043C08785992783FD79
:103750003FC080FD3DC09091AD0980911101891756
:10376000B8F5F1E08F1691F5222381F5F6018781F6
:10377000882371F58485882359F5808D8F3F11F05A
:103780008F5F808FF601808D863010F187898F5F83
:10379000878B843158F4868D42A16A2D8F700E94E8
:1037A000DB2FF601108E83E0878312C0F601868D31
:1037B00042A16A2D8F700E94DB2FF6018785816000
:1037C000878789818F5F0E94712602C0F601108E63
:1037D000F601878580FF05C08091B0098F5F8093D7
:1037E000B009F601878583FF05C08091AE098F5F20
:1037F0008093AE09F60187858111B39489818F5F2B
:103800008983823208F493CD7FC280913F04813056
:1038100009F0ADC119828981482F823208F074C243
:10382000242F332787E290E0289FB001299F700D55
:10383000389F700D1124FB01EB5BFB4F87858F7D5B
:10384000878787E2489FC00111240F2EF5E4CF2E11
:10385000F4E0DF2EF02DC80ED91EF601868D9927D3
:10386000807F9070803A910529F40F2EF1E4AF2EFD
:10387000F02D0CC0F601868D9927807F9070803BDB
:10388000910521F40F2EF2E4AF2EF02DF601848184
:1038900082FD4FC0808199278130910569F1803484
:1038A000910509F046C0818199278F30910561F01B
:1038B000803F9105F1F5868D42A16A2D8F700E949F
:1038C000902F8824839435C08981282F332787E25D
:1038D00090E0289FA001299F500D389F500D112482
:1038E000FA01EB5BFB4F868DF60142A16A2D8F70CA
:1038F0000E94DB2F88241DC0F601818199278F301B
:10390000910561F0803F9105A1F4868D42A16A2D59
:103910008F700E94902F882483940BC0F601868DAF
:1039200042A16A2D8F700E94DB2F8FE0F601818308
:103930008824F6018181803F09F057C084A18F3F20
:1039400009F453C00E94EB037C0100271127F60104
:10395000F6A2E5A289819927FC01ED58F64F8081F6
:103960009927AA27BB278E159F05A007B10724F02A
:10397000EE24FF2487010AC089819927FC01ED58B4
:10398000F64F8081E81AF10801091109F3E0EF16FA
:10399000F10401051105CCF089819927880F991F41
:1039A000FC01EB57F64F808191819C0144275527FC
:1039B000C801B7010E946E5520EE31E040E050E0B2
:1039C0000E94E25579018A0103C0EE24FF24870199
:1039D000F601F18AE08A8091AA099091AB098E0DD7
:1039E0009F1D9093AB098093AA09F6012089318924
:1039F000828993898217930780F58689813011F532
:103A000084899589892B69F5878588608787809166
:103A1000AE098F5F8093AE098081813059F4868D25
:103A200042A16A2D8F700E94DB2F88248FE0F6015F
:103A3000818382838981F601608971898F5F0E9409
:103A400039260FC081E0F601868B968185E0989F2C
:103A5000C0011124958B848B04C0F601168A158A47
:103A6000148AF601878D9927807F9070803A91059E
:103A700029F40F2EF1E49F2EF02D0CC0F601878D56
:103A80009927807F9070803B910521F40F2EF2E4FE
:103A90009F2EF02DF601878D42A1692D8F700E9417
:103AA0005E30282FF6018785992783FD42C080FD6F
:103AB00040C09091AD09809111018917D0F5F1E0D6
:103AC0008F16A9F5222399F5F6018781882389F5B8
:103AD0008485882371F58181803F59F5808D8F3FE2
:103AE00011F08F5F808FF601808D863010F187890D
:103AF0008F5F878B843158F4868D42A16A2D8F7039
:103B00000E94DB2FF601108E83E0878312C0F6013E
:103B1000868D42A16A2D8F700E94DB2FF60187856A
:103B20008160878789818F5F0E94712602C0F601BC
:103B3000108EF601878580FF05C08091B0098F5FE8
:103B40008093B009F601878583FF05C08091AE0997
:103B50008F5F8093AE09F60187858111B3948981C7
:103B60008F5F8983482F823208F45ACECDC080916E
:103B70003F04823009F0C8C019828981982F8232AF
:103B800008F0C2C087E2989FC00111240F2EF5E40F
:103B9000CF2EF4E0DF2EF02DC80ED91EF601868D53
:103BA0009927807F9070803A910529F40F2EF1E4D7
:103BB000AF2EF02D0CC0F601868D9927807F907076
:103BC000803B910521F40F2EF2E4AF2EF02D4091B1
:103BD000A9094423D1F0898199279C012F5F3F4F88
:103BE000842F99272817390741F4F601868D42A1C1
:103BF0006A2D8F700E94902F0FC0F601868D42A112
:103C00006A2D8F700E94DB2F07C0F601868D42A1BE
:103C10006A2D8F700E94902FF60184A18F3F09F4C6
:103C20006CC00E94EB037C0100271127F601F6A26D
:103C3000E5A280913E0480FF1CC089819927FC0188
:103C4000ED58F64F80819927AA27BB278E159F052F
:103C5000A007B10724F0EE24FF2487010AC0898160
:103C60009927FC01ED58F64F8081E81AF108010907
:103C70001109F3E0EF16F1040105110574F18091CB
:103C80003E0481FF19C089819927880F991FFC0183
:103C9000EB57F64F808191819C0144275527C8013D
:103CA000B7010E946E5520EE31E040E050E00E94E6
:103CB000E25579018A0114C0C801B70128EB31E04F
:103CC00040E050E00E946E5520EE31E040E050E0D0
:103CD0000E94E25579018A0103C0EE24FF24870186
:103CE000F601F18AE08A8091AA099091AB098E0DC4
:103CF0009F1D9093AB098093AA0989818F5F898367
:103D0000982F823208F43ECFBB2031F4B092AF0935
:103D1000B092B009B092B1090E941005982F80931B
:103D2000AC0980914004891710F4909340042091CD
:103D3000AA093091AB098091410490914204821705
:103D4000930720F4309342042093410421960FB648
:103D5000F894DEBF0FBECDBFDF91CF911F910F91C1
:103D6000FF90EF90DF90CF90BF90AF909F908F909B
:103D70000895815099270895CF93DF93EC01862F02
:103D80000E94B91E833278F4282F332787E290E00F
:103D9000289FA001299F500D389F500D1124FA0132
:103DA000EB5BFB4FC683DF91CF910895EF92FF92BB
:103DB0001F93CF937C01C0E080EC0E940A378111F1
:103DC000C1E081EC0E940A378111C26082EC0E943E
:103DD0000A378111C46081ED0E940A378111C860E1
:103DE00084EC0E940A378111C06185EC0E940A3779
:103DF0008111C06286EC0E940A378111C06487EC91
:103E00000E940A378111C06810E083EC0E940A37D3
:103E1000811111E082ED0E940A378111126083ED59
:103E20000E940A3781111460F701C0831183C0E03A
:103E300081E00E94ED0B8111C1E082E00E94ED0B58
:103E40008111C26083E00E94ED0B8111C46084E0A7
:103E50000E94ED0B8111C86085E00E94ED0B81117D
:103E6000C06186E00E94ED0B8111C06287E00E9474
:103E7000ED0B8111C06488E00E94ED0B8111C068D8
:103E8000F701C283C0E089E00E94ED0B8111C1E01F
:103E90008AE00E94ED0B8111C2608BE00E94ED0B65
:103EA0008111C4608CE00E94ED0B8111C8608DE02F
:103EB0000E94ED0B8111C0618EE00E94ED0B81111B
:103EC000C0628FE00E94ED0B8111C06480E10E940E
:103ED000ED0B8111C068F701C383C0E081E10E944E
:103EE000ED0B8111C1E082E10E94ED0B8111C260F6
:103EF00083E10E94ED0B8111C46084E10E94ED0B0F
:103F00008111C86085E10E94ED0B8111C06186E1DD
:103F10000E94ED0B8111C06287E10E94ED0B8111BF
:103F2000C06488E10E94ED0B8111C068F701C48371
:103F3000C0E089E10E94ED0B8111C1E08AE10E949D
:103F4000ED0B8111C2608BE10E94ED0B8111C46009
:103F50008CE10E94ED0B8111C8608DE10E94ED0B98
:103F60008111C0618EE10E94ED0B8111C0628FE171
:103F70000E94ED0B8111C06480E20E94ED0B811163
:103F8000C068F701C583CF911F91FF90EF9008950E
:103F90001F93CF93DF93182FEB010E94B91E482F78
:103FA000833218F080E090E073C0992727E230E078
:103FB000829FB001839F700D929F700D1124FB01B1
:103FC000E75BFB4F208122FD24C0FB01EB5BFB4F35
:103FD0008181803F71F485859685892B39F421FD97
:103FE00005C020FD03C0878585FF03C08FE088835F
:103FF00035C0242F332787E290E0289FF001299FC6
:10400000F00D389FF00D1124EB5BFB4F818188830D
:1040100025C030E0232F5DE0259FC0011124DC0185
:10402000AC51B64FFD018181813099F490E07FE081
:1040300060EFFD01E90FF11D8185841739F431E04E
:104040008C9182FF02C0788301C068839F5F9430A7
:1040500080F32F5F253010F43323F1F2242F332720
:1040600087E290E0289FA001299F500D389F500DB6
:104070001124FA01EB5BFB4F878589838089918945
:104080009C838B83812F0E94BC268A8381E090E0F1
:10409000DF91CF911F9108950E94B91E833218F0CD
:1040A00080E090E00895282F332787E290E0289F52
:1040B000A001299F500D389F500D1124FA01EB5B90
:1040C000FB4F8181803F59F4FA01E75BFB4F208170
:1040D00021FD05C020FD03C081E090E0089580E04F
:1040E00090E008950E94B91E833218F080E090E0BD
:1040F0000895282F332787E290E0289FA001299F69
:10410000500D389F500D1124FA01EB5BFB4F2785B2
:10411000283011F0213019F481E090E0089580E01A
:1041200090E00895FC018091AA099091AB099183D8
:1041300080838091AC0982838091AD0983838091D3
:10414000AE0984838091AF0985838091B00986830D
:104150008091B109878308959EEF81B1892381B948
:1041600082B1892382B917B818B891EF8AB189232F
:104170008AB98BB189238BB908950F930E94B91E18
:10418000282F833168F000E0202F40E050E06AEDF6
:1041900079E082E191E00E94C62380E090E007C0D0
:1041A00083E799E0FC01E20FF11D808199270F91CF
:1041B00008950F930E94B91E833168F000E0202F0C
:1041C00040E050E068EE79E082E191E00E94C62391
:1041D00080E692E212C09927880F991FFC01EB57E5
:1041E000F64F2081318184E190E0289FA001299F32
:1041F000500D389F500D1124CA010F9108950F934F
:10420000CF93DF93EB010E94B91E833158F000E099
:10421000202F40E050E067EF79E082E191E00E94DA
:10422000C62312C0992725E839E0880F991FFC01A1
:10423000E20FF31FCE0164E170E00E949955718393
:104240006083C9010E94A529DF91CF910F91089544
:104250000E94B91E833118F080E090E00895282F65
:10426000332787E290E0289FA001299F500D389FB7
:10427000500D1124FA01EB5BFB4F80899189089561
:104280000E94B91E833118F080E090E00895282F35
:10429000332787E290E0289FA001299F500D389F87
:1042A000500D1124FA01EB5BFB4F85A196A10895F7
:1042B00080933E046093A90908951F93CF93C0E0B3
:1042C00017E2C19FC0011124FC01EB5BFB4F84A1ED
:1042D0008F3F41F00E94EB032C2F3327F901ED585B
:1042E000F64F8083CF5FC23160F383E799E00E948D
:1042F0008529CF911F910895CF9380913F048330FA
:1043000059F083E080933F04C0E061E08C2F0E946D
:104310000E12CF5FC232C8F3CF9108958091DD09AC
:10432000882341F00E949B210E94C62186EB99E0E0
:104330000E9413220895259A2D98269A2E988AEA8B
:104340008093800089E18093810010928500109213
:10435000840080E395E0909387008093860010921C
:1043600089001092880010928B0010928A0010929F
:104370008D0010928C0060E070E081E00E94F121DD
:1043800060E070E082E00E94F121089510929000B8
:1043900084E0809391001092950010929400109206
:1043A0009700109296001092990010929800109227
:1043B0009B0010929A0010929D0010929C00109207
:1043C000B3091092B2091092B5091092B409809104
:1043D000690088608093690010926A00E99AE19A06
:1043E000089599278230910581F0833091051CF45E
:1043F000019721F00895039779F00895872F992761
:1044000080938900609388000895872F992780936F
:104410008B0060938A000895872F992780938D00E1
:1044200060938C000895FC01118210821382128225
:1044300085E090E09583848316820895EF92FF9241
:104440000F931F93CF93DF93EC018E81982F8F5F93
:104450008E83963068F060E375E081E00E94F12180
:1044600060E375E082E00E94F12186E08E8355C012
:104470008A819B819C0144275527888199817C01F1
:1044800000271127DA01C901689412F8880F991FD3
:10449000AA1FBB1F1694D1F7820F931FA41FB51F2D
:1044A000280F391F4A1F5B1FCA01B90125E830E0F8
:1044B00040E050E00E946E55A80197010E94C0554F
:1044C000E901C901845490408652944010F0C0E341
:1044D000D5E08091DD09882349F080910905803F6E
:1044E00029F4BE0181E00E94F12105C060E375E07E
:1044F00081E00E94F1218091DE09882349F08091BA
:104500004106803F29F4BE0182E00E94F12105C0EE
:1045100060E375E082E00E94F121DF91CF911F916D
:104520000F91FF90EF9008951F920F920FB60F9288
:1045300011242F933F938F939F9380919400282F62
:104540003327322F2227809195009927282B392B4A
:104550008091690099278C7090700C97E1F43093EA
:10456000B7092093B609109294001092950080919B
:104570004304909144049093B9098093B809109230
:104580004404109243041092BC09809169008B7F0F
:104590008093690010C08091690099278C70907099
:1045A000089749F4309344042093430480916900B0
:1045B0008460809369009F918F913F912F910F901C
:1045C0000FBE0F901F901895CF93DF93CDB7DEB736
:1045D00023970FB6F894DEBF0FBECDBFFE01319614
:1045E000A0E8B1E083E090E021E08030920719F488
:1045F0000E943C5603C0182E0E943C5643E050E0F7
:1046000060E271E0CE0101960E949644882391F009
:104610000E942423E0E2F1E0A0E8B1E083E090E032
:1046200021E08030920719F40E944D5603C0182EE5
:104630000E944D56279823960FB6F894DEBF0FBE02
:10464000CDBFDF91CF910895CF93DF93CDB7DEB784
:104650006E970FB6F894DEBF0FBECDBF84E1FE01AA
:104660003B9611928A95E9F740E064E124E130E05D
:10467000522FFE013B96469FC0011124DC01AC572E
:10468000BE4F2115310551F081E02030380719F473
:104690000E944D5603C0152E0E944D56A8954F5F9F
:1046A000483038F31982FE013196A3E8B1E081E089
:1046B00090E021E08030920719F40E944D5603C02B
:1046C000182E0E944D566E960FB6F894DEBF0FBEA0
:1046D000CDBFDF91CF910895CF93DF93CDB7DEB7F4
:1046E00021970FB6F894DEBF0FBECDBFFE01319605
:1046F000A3E8B1E081E090E021E08030920719F476
:104700000E943C5603C0182E0E943C568981893075
:1047100010F088E089838981992721960FB6F89453
:10472000DEBF0FBECDBFDF91CF910895CF93DF9352
:10473000CDB7DEB764970FB6F894DEBF0FBECDBF1E
:104740009B01FE01319694E1899FD0011124A0596B
:10475000BE4F84E190E041E08030940719F40E945C
:104760003C5603C0182E0E943C5684E1FE0131964F
:10477000D90101900D928A95E1F764960FB6F894ED
:10478000DEBF0FBECDBFDF91CF9108956F927F92B4
:104790008F929F92AF92BF92CF92DF92EF92FF9251
:1047A0000F931F93CF93DF93CDB7DEB7A9970FB6C3
:1047B000F894DEBF0FBECDBF6C015B013A01022F42
:1047C000FE01B996A3E8B1E081E090E021E08030FD
:1047D000920719F40E943C5603C0182E0E943C56C2
:1047E00089A5883008F0D4C09924FE01759684E12B
:1047F000DF011D928A95E9F7B601CF010E94675546
:10480000192D89A5981608F05EC00F2EF4E18F2EA1
:10481000F02D0F2EF4E1EF2EFF24F02DFE01319646
:10482000189DC0011124DC01AC57BE4FE114F10406
:1048300059F020E0E21621E0F20619F40E943C56FD
:1048400003C01E2C0E943C568D859E858A159B05B3
:1048500099F546E050E0B601CE0101960E949644DB
:10486000882351F5992493948F858A3008F090C05D
:10487000890D8F87053008F004E0198A1A8A1B8A8F
:104880001C8A802F9927AC01B301CE0141960E946A
:104890005055FE013196189DD0011124AC57BE4FE2
:1048A00084E190E021E08030920719F40E944D5697
:1048B00003C0182E0E944D561F5F89A5181718F4C3
:1048C000992009F4ABCF992009F052C089A588300E
:1048D00008F04EC08F5F89A78CE0FE0131961192DF
:1048E0008A95E9F7F60101900020E9F731972E2F1C
:1048F0002C192C3008F02BE010E0121780F4AE01D8
:104900004F5F5F4F812F9927DC01A40FB51FF60180
:10491000E80FF91F80818C931F5F121798F3BE86F2
:10492000AD8681E08F87053008F004E0088B198A96
:104930001A8A1B8A1C8A802F9927AC01B301CE01E9
:1049400041960E945055FE01319699A584E1989FA9
:10495000D0011124A059BE4F84E190E021E08030C5
:10496000920719F40E944D5603C0182E0E944D560E
:10497000FE01B996A3E8B1E081E090E021E080304B
:10498000920719F40E944D5603C0182E0E944D56EE
:10499000A9960FB6F894DEBF0FBECDBFDF91CF91C1
:1049A0001F910F91FF90EF90DF90CF90BF90AF904D
:1049B0009F908F907F906F900895089582E1EDEE23
:1049C000FEE011928A95E9F780E1EFEFFEE01192A7
:1049D0008A95E9F7E1E2FFE0A8E8B0E082E190E043
:1049E00021E08030920719F40E943C5603C0182E33
:1049F0000E943C56E3E3FFE0AAE9B0E082E190E0E8
:104A000021E08030920719F40E943C5603C0182E12
:104A10000E943C56E5E4FFE0ACEAB0E080E190E0C3
:104A200021E08030920719F40E943C5603C0182EF2
:104A30000E943C56EFE0FFE0ADEBB0E082E190E099
:104A400021E08030920719F40E943C5603C0182ED2
:104A50000E943C56E5E2FAE0A5E8B0E081E090E093
:104A600021E08030920719F40E943C5603C0182EB2
:104A70000E943C56E6E2FAE0A6E8B0E082E090E070
:104A800021E08030920719F40E943C560895182EB8
:104A90000E943C560895CF93DF93CDB7DEB762975F
:104AA0000FB6F894DEBF0FBECDBFFE01319682E196
:104AB000DF011D928A95E9F7A8E8B0E082E190E075
:104AC00021E08030920719F40E944D5603C0182E41
:104AD0000E944D56FE013196AAE9B0E082E190E0D5
:104AE00021E08030920719F40E944D5603C0182E21
:104AF0000E944D56FE013196ACEAB0E080E190E0B4
:104B000021E08030920719F40E944D5603C0182E00
:104B10000E944D56FE013196ADEBB0E082E190E08F
:104B200021E08030920719F40E944D5603C0182EE0
:104B30000E944D560E94DE2462960FB6F894DEBFA6
:104B40000FBECDBFDF91CF9108950E94AF12982F75
:104B50008091250A891790F49093250AE5E2FAE0FE
:104B6000A5E8B0E081E090E021E08030920719F400
:104B70000E944D5603C0182E0E944D560E94AA1244
:104B80009C018091260A9091270A82179307A0F42E
:104B90003093270A2093260AE6E2FAE0A6E8B0E07E
:104BA00082E090E021E08030920719F40E944D5697
:104BB0000895182E0E944D5608958091250A992730
:104BC00008958091260A9091270A089590E04DEE6D
:104BD0005EE0292F3327F901E40FF51F808180FF64
:104BE00017C08E7F8083D901A857BF4FF901EF5DB1
:104BF000F04F8081082E0E944156D901A656BF4F22
:104C0000F901ED5CF04F8081082E0E944156089515
:104C1000E92FFF27DF01A40FB51F8C9181FF0CC086
:104C20008D7F8C93DF01A354BF4FE15FF04F8081F4
:104C3000082E0E94415608959F5F923150F290E0F5
:104C40002FEF3EE0E92FFF27DF01A20FB31F8C916A
:104C5000813059F41C92DF01A455BF4FEB5BF04F3C
:104C60008081082E0E94415608959F5F903150F335
:104C70000895282F2150223198F581E29FE0FC0110
:104C8000E20FF11D3081832F9927929582958F70C5
:104C900089279F7089278F30910514F5482F4F5F22
:104CA000942F9295907F832F8F70890F8083CB01F3
:104CB00083709070892B11F041E001C040E03327F0
:104CC000F901ED5CF04FCB01969587959695879508
:104CD000840F8083F901E351F14F808181608083EB
:104CE0000895E82FE150E231C0F4FF27DF01AF5D06
:104CF000B04F2C91822F99278F7090700F971CF5D1
:104D0000822F8F708F5F922F907F890F8C93E3514A
:104D1000F14F80818160808308958351803198F4C0
:104D2000E82FFF27DF01AB5BB04F2C91822F992733
:104D30008F7090700F973CF4822F8F5F8C93E150AF
:104D4000F14F81E08083089581508231A0F4E82FF3
:104D5000FF27DF01A15FB04F2C91822F99278F7021
:104D600090700F9744F4822F8F5F8C93E351F14F33
:104D70008081826080830895E82FE150E23188F4D9
:104D80002E2F3327F901EF5DF04F8081882331F416
:104D9000F901E15FF04F8081882391F081E090E09C
:104DA0000895282F2351203158F485E49FE0FC0119
:104DB000E20FF11D8081882319F081E090E00895D1
:104DC00080E090E00895CF93DF93EC01FC0120E5B3
:104DD00032E08EE090E041E08030940721F4D90188
:104DE0000E944D5604C0D901182E0E944D56CE0186
:104DF0000296AC01698188810E94B312DF91CF9144
:104E00000895FC01A0E5B2E08EE090E021E0803062
:104E1000920719F40E943C560895182E0E943C56A1
:104E20000895FC01A0E6B2E081E190E021E080304D
:104E3000920719F40E944D560895182E0E944D565F
:104E40000895FC01A0E6B2E081E190E021E080302D
:104E5000920719F40E943C560895182E0E943C5661
:104E60000895FC01A0EABBE088E090E021E08030FA
:104E7000920719F40E944D560895182E0E944D561F
:104E80000895FC01A0EABBE088E090E021E08030DA
:104E9000920719F40E943C560895182E0E943C5621
:104EA00008950F93CF93DF93CDB7DEB721970FB659
:104EB000F894DEBF0FBECDBF8983853060F000E07F
:104EC00021E0AE014F5F5F4F67E470E084E291E064
:104ED0000E94C62315C0898198E1899FC0011124D1
:104EE000FB01DC01AE5FB04F88E190E021E0803053
:104EF000920719F40E944D5603C0182E0E944D5679
:104F000021960FB6F894DEBF0FBECDBFDF91CF91D3
:104F10000F9108950F93CF93DF93CDB7DEB721970D
:104F20000FB6F894DEBF0FBECDBF8983853060F029
:104F300000E021E0AE014F5F5F4F64E570E084E286
:104F400091E00E94C62315C0898198E1899FC00124
:104F50001124FB01DC01AE5FB04F88E190E021E05D
:104F60008030920719F40E943C5603C0182E0E940C
:104F70003C5621960FB6F894DEBF0FBECDBFDF9131
:104F8000CF910F9108950F93CF93DF93CDB7DEB7F5
:104F900021970FB6F894DEBF0FBECDBF8983803254
:104FA00060F000E021E0AE014F5F5F4F60E670E02F
:104FB00084E291E00E94C62314C0FB0199818CE237
:104FC000989FD0011124A058BC4F8CE290E021E0C2
:104FD0008030920719F40E944D5603C0182E0E948B
:104FE0004D5621960FB6F894DEBF0FBECDBFDF91B0
:104FF000CF910F9108950F93CF93DF93CDB7DEB785
:1050000021970FB6F894DEBF0FBECDBF89838032E3
:1050100060F000E021E0AE014F5F5F4F6AE670E0B4
:1050200084E291E00E94C62314C0FB0199818CE2C6
:10503000989FD0011124A058BC4F8CE290E021E051
:105040008030920719F40E943C5603C0182E0E942B
:105050003C5621960FB6F894DEBF0FBECDBFDF9150
:10506000CF910F9108950F93CF93DF93CDB7DEB714
:1050700021970FB6F894DEBF0FBECDBF8983843170
:1050800060F000E021E0AE014F5F5F4F64E770E049
:1050900084E291E00E94C62314C0FB01998188E15B
:1050A000989FD0011124A05FB64F88E190E021E0E5
:1050B0008030920719F40E944D5603C0182E0E94AA
:1050C0004D5621960FB6F894DEBF0FBECDBFDF91CF
:1050D000CF910F9108950F93CF93DF93CDB7DEB7A4
:1050E00021970FB6F894DEBF0FBECDBF8983843100
:1050F00060F000E021E0AE014F5F5F4F6EE770E0CF
:1051000084E291E00E94C62314C0FB01998188E1EA
:10511000989FD0011124A05FB64F88E190E021E074
:105120008030920719F40E943C5603C0182E0E944A
:105130003C5621960FB6F894DEBF0FBECDBFDF916F
:10514000CF910F910895CF93DF93CDB7DEB76997D5
:105150000FB6F894DEBF0FBECDBFFC01862F815085
:10516000823218F080E090E02AC06150808189830B
:1051700081818A8382818B8383818C8387818887E5
:105180008789888F808D898F848195819E838D8387
:1051900086818F83DF0118968FE0FE0139960D908E
:1051A00001928A95E1F789E1689FC0011124805539
:1051B000944FBC01CE0101960E94742999276996EB
:1051C0000FB6F894DEBF0FBECDBFDF91CF9108952B
:1051D0000F931F93CF93DF93CDB7DEB769970FB6C9
:1051E000F894DEBF0FBECDBF8C01962F9150923246
:1051F000B0F589E1989FC00111249E012F5F3F4FB8
:10520000DC01A055B44F89E190E041E08030940783
:1052100021F4F9010E943C5604C0F901182E0E94A5
:105220003C568981F80180838A8181838B818283C6
:105230008C81838388858783888D878B898D808FF8
:105240008D819E81958384838F818683D801189672
:105250008FE0FE01399601900D928A95E1F76996EB
:105260000FB6F894DEBF0FBECDBFDF91CF911F9177
:105270000F91089581508B30C8F4FB01A82FBB27F4
:10528000CD0182959295907F9827807F9827DC01A9
:10529000A051B54F80E190E021E08030920719F4F1
:1052A0000E944D560895182E0E944D560895815023
:1052B0008B30C8F4FB01A82FBB27CD0182959295B6
:1052C000907F9827807F9827DC01A051B54F80E11F
:1052D00090E021E08030920719F40E943C56089536
:1052E000182E0E943C560895FC01DB0189E190E0F4
:1052F00021E08030920719F40E944D5603C0182E09
:105300000E944D5681E090E00895FC01A0E1B0E0DC
:1053100082E190E021E08030920719F40E944D561E
:105320000895182E0E944D560895FC01A0E1B0E0AA
:1053300082E190E021E08030920719F40E943C560F
:105340000895182E0E943C560895FC01A0E3B0E099
:1053500084E290E021E08030920719F40E944D56DB
:105360000895182E0E944D560895FC01A0E3B0E068
:1053700084E290E021E08030920719F40E943C56CC
:105380000895182E0E943C560895FC01A0E8B2E052
:1053900088E190E021E08030920719F40E944D5698
:1053A0000895182E0E944D560895FC01A0E8B2E021
:1053B00088E190E021E08030920719F40E943C5689
:1053C0000895182E0E943C5608950F93FC01808189
:1053D000882319F488E992E016C08081813019F49D
:1053E0008EED92E010C08081823019F484E293E067
:1053F0000AC000E021E0AF0167E471E084E291E0DF
:105400000E94C6230DC0DC0186E490E021E08030DC
:10541000920719F40E944D5603C0182E0E944D5653
:105420000F9108950F93CF93DF93CDB7DEB72197F8
:105430000FB6F894DEBF0FBECDBF8983882319F461
:1054400088E992E018C08981813019F48EED92E0EC
:1054500012C08981823019F484E293E00CC000E02C
:1054600021E0AE014F5F5F4F60E671E084E291E0C2
:105470000E94C6230EC0FB01DC0186E490E021E01F
:105480008030920719F40E943C5603C0182E0E94E7
:105490003C5621960FB6F894DEBF0FBECDBFDF910C
:1054A000CF910F910895CF93DF93CDB7DEB760977B
:1054B0000FB6F894DEBF0FBECDBFFE013196A0E05F
:1054C000B0E080E190E021E08030920719F40E9482
:1054D0003C5603C0182E0E943C568B858F3119F420
:1054E0008FE190E008C08B85803219F480E290E073
:1054F00002C08FE190E060960FB6F894DEBF0FBE59
:10550000CDBFDF91CF910895CFEDD0E1DEBFCDBF0C
:1055100082E89FE09093560F8093550F88E190E0CA
:105520009093560F8093550F89E190E09093560F1A
:105530008093550F80E190E09093560F8093550F24
:105540000E9492430E948A2D0E94D5120E947A05E1
:105550000E94A4430E9430380E94E422FE0131964A
:10556000A0E0B0E084E090E021E08030920719F400
:105570000E943C5603C0182E0E943C5644E050E066
:1055800068E371E0CE0101960E9496448823C1F140
:105590008E010F5F1F4F80E2D8011D928A95E9F7B7
:1055A00085E0E8E3F1E0D80101900D928A95E1F7FA
:1055B0001D821E821F82188619861A861B860E94EB
:1055C000EF15F801A0E0B0E080E190E021E080304C
:1055D000920719F40E944D5603C0182E0E944D5692
:1055E000FE013196A0E0B0E084E090E021E0803060
:1055F000920719F40E944D5603C0182E0E944D5672
:10560000FE013196A0E3B2E08AE090E021E0803034
:10561000920719F40E943C5603C0182E0E943C5673
:105620004AE050E064E571E0CE0101960E949644A4
:10563000882369F10E940F160E947E0B0E945B4630
:105640000E944F06FE01319680E2DF011D928A958D
:10565000E9F7A2E8BFE080E190E021E08030920726
:1056600019F40E944D5603C0182E0E944D56E4E5D1
:10567000F1E0A0E3B2E08AE090E021E08030920720
:1056800019F40E944D5603C0182E0E944D56FE017B
:105690003196A0E8B1E083E090E021E0803092070D
:1056A00019F40E943C5603C0182E0E943C5643E059
:1056B00050E06DE371E0CE0101960E94964488238C
:1056C00091F00E942423EDE3F1E0A0E8B1E083E053
:1056D00090E021E08030920719F40E944D5603C0FB
:1056E000182E0E944D56FE013196A0E8B0E085E0EC
:1056F00090E021E08030920719F40E943C5603C0EC
:10570000182E0E943C5645E050E061E471E0CE0165
:1057100001960E949644882309F475C0FE013196D3
:1057200080E2DF011D928A95E9F7ACEBB0E081E001
:1057300090E021E08030920719F40E944D5603C09A
:10574000182E0E944D56FE013196A5E8B0E081E08A
:1057500090E021E08030920719F40E944D5603C07A
:10576000182E0E944D56FE013196A6E8B0E082E068
:1057700090E021E08030920719F40E944D5603C05A
:10578000182E0E944D56FE013196A8E8B0E082E145
:1057900090E021E08030920719F40E944D5603C03A
:1057A000182E0E944D56FE013196ACEAB0E080E121
:1057B00090E021E08030920719F40E944D5603C01A
:1057C000182E0E944D56FE013196ADEBB0E082E1FD
:1057D00090E021E08030920719F40E944D5603C0FA
:1057E000182E0E944D56E1E4F1E0A0E8B0E085E01B
:1057F00090E021E08030920719F40E944D5603C0DA
:10580000182E0E944D560E944E0A0E949C300E9403
:1058100018460E94FD160E94773787E00E94CC4F01
:1058200078940E94EE41A89580E00E948C370E94F7
:105830003B38FACF1F93162FA39899278770907043
:10584000880F991F81640E949D43812F0E949D4370
:1058500080E00E949D43A39A99271F9108950F937A
:105860001F93162F042FA398992787709070880F85
:10587000991F80640E949D43812F0E949D43802F29
:105880000E949D43A39A1F910F9108951F93CF9358
:10589000C091280ACC2389F511E01093280A4CE125
:1058A0006AE08C2F0E942F2C4C2F6C2F8C2F0E9483
:1058B0002F2C4FEF612F8C2F0E942F2C4C2F62E04A
:1058C0008C2F0E942F2C4C2F63E08C2F0E942F2CAA
:1058D0004C2F64E08C2F0E942F2C4C2F65E08C2FD6
:1058E0000E942F2C4C2F6CE08C2F0E942F2C4C2FC1
:1058F0006DE08C2F0E942F2C0AC1C091280AC13064
:1059000089F54CE16AE08C2F0E942F2C40E0642F37
:105910008C2F0E942F2C4FEF6C2F8C2F0E942F2C3E
:1059200040E062E08C2F0E942F2C40E063E08C2F3F
:105930000E942F2C40E064E08C2F0E942F2C40E02E
:1059400065E08C2F0E942F2C40E06CE08C2F0E9491
:105950002F2C40E06DE08C2F0E942F2C82E0809352
:10596000280AD5C0C091280AC23089F54CE16AE006
:105970008C2F0E942F2C40E0642F8C2F0E942F2C04
:105980004FEF61E08C2F0E942F2C40E06C2F8C2F6A
:105990000E942F2C40E063E08C2F0E942F2C40E0CF
:1059A00064E08C2F0E942F2C40E065E08C2F0E9439
:1059B0002F2C40E06CE08C2F0E942F2C40E06DE0FB
:1059C0008C2F0E942F2C83E08093280AA0C0C091C6
:1059D000280AC33089F54CE16AE08C2F0E942F2CF5
:1059E00040E0642F8C2F0E942F2C4FEF61E08C2F12
:1059F0000E942F2C40E062E08C2F0E942F2C40E070
:105A00006C2F8C2F0E942F2C40E064E08C2F0E9482
:105A10002F2C40E065E08C2F0E942F2C40E06CE0A2
:105A20008C2F0E942F2C40E06DE08C2F0E942F2C99
:105A300084E08093280A6BC0C091280AC43089F59D
:105A40004CE16AE08C2F0E942F2C4CEF60E08C2FF1
:105A50000E942F2C4FEF61E08C2F0E942F2C40E0F2
:105A600062E08C2F0E942F2C40E063E08C2F0E947C
:105A70002F2C40E06C2F8C2F0E942F2C40E065E0F3
:105A80008C2F0E942F2C40E06CE08C2F0E942F2C3A
:105A900040E06DE08C2F0E942F2C85E08093280A37
:105AA00036C0C091280AC53081F54CE16AE08C2FE0
:105AB0000E942F2C40E0642F8C2F0E942F2C40EF4F
:105AC00061E08C2F0E942F2C40E062E08C2F0E941E
:105AD0002F2C40E063E08C2F0E942F2C40E064E0EC
:105AE0008C2F0E942F2C40E06C2F8C2F0E942F2C8B
:105AF00040E06CE08C2F0E942F2C40E06DE08C2F5A
:105B00000E942F2C1092280A02C01092280ACF91CE
:105B10001F9108959B9AA39A4CE16AE080E00E944D
:105B20002F2C40E064E1842F0E942F2C40E0642F52
:105B3000842F0E942F2C4FEF61E080E00E942F2CD9
:105B400040E062E0842F0E942F2C40E063E0842F2D
:105B50000E942F2C40E064E0842F0E942F2C40E014
:105B600065E0842F0E942F2C40E06CE0842F0E947F
:105B70002F2C40E06DE0842F0E942F2C4CE16AE036
:105B800081E00E942F2C40E064E181E00E942F2CF4
:105B900040E0642F81E00E942F2C4FEF61E0862FC0
:105BA0000E942F2C40E062E081E00E942F2C40E018
:105BB00063E081E00E942F2C40E064E081E00E94DD
:105BC0002F2C40E065E081E00E942F2C40E06CE04B
:105BD00081E00E942F2C40E06DE081E00E942F2C9C
:105BE0004CE16AE082E00E942F2C40E064E182E018
:105BF0000E942F2C40E0642F82E00E942F2C4FEF58
:105C000061E082E00E942F2C40E062E0862F0E943B
:105C10002F2C40E063E082E00E942F2C40E064E003
:105C200082E00E942F2C40E065E082E00E942F2C51
:105C300040E06CE082E00E942F2C40E06DE082E0CA
:105C40000E942F2C4CE16AE083E00E942F2C40E060
:105C500064E183E00E942F2C40E0642F83E00E94E7
:105C60002F2C4FEF61E083E00E942F2C40E062E098
:105C700083E00E942F2C40E063E0862F0E942F2CAF
:105C800040E064E083E00E942F2C40E065E083E088
:105C90000E942F2C40E06CE083E00E942F2C40E01B
:105CA0006DE083E00E942F2C4CE16AE084E00E94CA
:105CB0002F2C40E064E184E00E942F2C4CEF60E048
:105CC00084E00E942F2C4FEF61E084E00E942F2C93
:105CD00040E062E084E00E942F2C40E063E084E03A
:105CE0000E942F2C40E064E0862F0E942F2C40E081
:105CF00065E084E00E942F2C40E06CE084E00E948C
:105D00002F2C40E06DE084E00E942F2C4CE16AE0F3
:105D100085E00E942F2C40E064E185E00E942F2C5A
:105D200040E065E185E00E942F2C40E0642F85E093
:105D30000E942F2C40EF61E085E00E942F2C40E074
:105D400062E085E00E942F2C40E063E085E00E9445
:105D50002F2C40E064E085E00E942F2C40E065E0BD
:105D6000862F0E942F2C40E06CE085E00E942F2CB3
:105D700040E06DE085E00E942F2C08950F931F9363
:105D8000CF93082FC62F142F20E030E0613611F496
:105D900021E030E080E090E0C13411F481E090E057
:105DA000822B932B892B91F060E0812F0E941A2C7B
:105DB00021E030E0002E02C0220F331F0A94E2F7E8
:105DC000482F422B60E0812F0E942F2C20E030E0F2
:105DD000C23611F421E030E080E090E0C23411F4EA
:105DE00081E090E0822B932B892B89F061E0812F59
:105DF0000E941A2C21E030E002C0220F331F0A95C6
:105E0000E2F7482F422B61E0812F0E942F2CCF9187
:105E10001F910F9108950F931F93CF93082FC62FB3
:105E2000142F20E030E0613611F421E030E080E012
:105E300090E0C13411F481E090E0822B932B892B08
:105E4000A1F060E0812F0E941A2C21E030E0002EAA
:105E500002C0220F331F0A94E2F7922F9095482F29
:105E6000492360E0812F0E942F2C20E030E0C236D1
:105E700011F421E030E080E090E0C23411F481E0E0
:105E800090E0822B932B892B99F061E0812F0E9467
:105E90001A2C21E030E002C0220F331F0A95E2F7EE
:105EA000922F9095482F492361E0812F0E942F2C3B
:105EB000CF911F910F9108950F931F93CF93182F98
:105EC000C62F042F20E030E0613611F421E030E0ED
:105ED00080E090E0C13411F481E090E0822B932BBC
:105EE000892B29F0412F64E1802F0E942F2C20E084
:105EF00030E0C23611F421E030E080E090E0C234BE
:105F000011F481E090E0822B932B892B29F0412F13
:105F100065E1802F0E942F2CCF911F910F91089542
:105F20000F931F93CF93082FC62F142F50E020E01C
:105F300030E0613611F421E030E080E090E0C134DF
:105F400011F481E090E0822B932B892B71F062E1B8
:105F5000812F0E941A2C21E030E0002E02C0220F77
:105F6000331F0A94E2F7582F522B20E030E0C2365C
:105F700011F421E030E080E090E0C23411F481E0DF
:105F800090E0822B932B892B69F063E1812F0E9493
:105F90001A2C21E030E002C0220F331F0A95E2F7ED
:105FA000582F522B412F6C2F852F0E945C2FCF91A1
:105FB0001F910F9108950F931F93CF93082FC62F12
:105FC000142F50E020E030E0613611F421E030E0A1
:105FD00080E090E0C13411F481E090E0822B932BBB
:105FE000892B81F062E1812F0E941A2C21E030E0A0
:105FF000002E02C0220F331F0A94E2F7922F9095D1
:10600000582F592320E030E0C23611F421E030E06F
:1060100080E090E0C23411F481E090E0822B932B79
:10602000892B79F063E1812F0E941A2C21E030E066
:1060300002C0220F331F0A95E2F7922F9095582F36
:106040005923412F6C2F852F0E945C2FCF911F91D8
:106050000F9108951F93CF93C82F162F40E020E093
:1060600030E0813611F421E030E080E090E0C1348E
:1060700011F481E090E0822B932B892B29F062E1CF
:10608000812F0E941A2C482F20E030E0C23611F4F4
:1060900021E030E080E090E0C23411F481E090E053
:1060A000822B932B892B29F063E1812F0E941A2CDC
:1060B000482F842F9927CF911F9108950F931F93F5
:1060C000CF93182FC62F042F40E020E030E0613638
:1060D00011F421E030E080E090E0C13411F481E07F
:1060E00090E0822B932B892B29F062E1802F0E9474
:1060F0001A2C482F20E030E0C23611F421E030E0C5
:1061000080E090E0C23411F481E090E0822B932B88
:10611000892B29F063E1802F0E941A2C482F81E0FF
:1061200090E002C0880F991F1A95E2F784239927FF
:10613000CF911F910F9108950E94A60E86E89AE0D4
:1061400090931D0B80931C0B10921E0B1092150B3D
:106150001092160B85E19BE00E94B70E8823D1F7C1
:106160001092140B8EE89AE09093290B8093280BE1
:1061700010922A0B1092210B1092220B81E29BE0CD
:106180000E94B70E8823D1F71092200B86E99AE07F
:106190009093350B8093340B1092360B10922D0B8D
:1061A00010922E0B8DE29BE00E94B70E8823D1F750
:1061B00010922C0B8EE99AE09093410B8093400B48
:1061C0001092420B1092390B10923A0B89E39BE02C
:1061D0000E94B70E8823D1F71092380B86E39AE01D
:1061E0009093AE0A8093AD0A1092AF0A1092A60A5D
:1061F00082E08093A70A86EA9AE00E94B70E88237D
:10620000D1F78EE39AE09093B90A8093B80A10927E
:10621000BA0A1092B10A82E08093B20A81EB9AE046
:106220000E94B70E8823D1F786E49AE09093C40ABF
:106230008093C30A1092C50A1092BC0A82E0809330
:10624000BD0A8CEB9AE00E94B70E8823D1F78EE44A
:106250009AE09093CF0A8093CE0A1092D00A1092BF
:10626000C70A82E08093C80A87EC9AE00E94B70EC2
:106270008823D1F786E59AE09093DA0A8093D90AC9
:106280001092DB0A1092D20A82E08093D30A82ED48
:106290009AE00E94B70E8823D1F78EE59AE090939A
:1062A000E50A8093E40A1092E60A1092DD0A82E081
:1062B0008093DE0A8DED9AE00E94B70E8823D1F715
:1062C00086E69AE09093F00A8093EF0A1092F10A22
:1062D0001092E80A82E08093E90A88EE9AE00E9430
:1062E000B70E8823D1F78EE69AE09093FB0A80934D
:1062F000FA0A1092FC0A1092F30A82E08093F40AE0
:1063000083EF9AE00E94B70E8823D1F786E79AE0E0
:106310009093060B8093050B1092070B1092FE0AC8
:1063200082E08093FF0A8EEF9AE00E94B70E8823E6
:10633000D1F78EE79AE09093110B8093100B109297
:10634000120B1092090B82E080930A0B89E09BE00C
:106350000E94B70E8823D1F708958091140B8823EB
:10636000E1F08091140B813059F484E19BE00196B7
:106370000E94B70E882389F482E08093140B0DC02D
:106380008091140B823049F484E19BE001960E94D5
:10639000C90F882311F48093140B8091200B88235C
:1063A000E1F08091200B813059F480E29BE001966E
:1063B0000E94B70E882389F482E08093200B0DC0E1
:1063C0008091200B823049F480E29BE001960E948C
:1063D000C90F882311F48093200B80912C0B882304
:1063E000E1F080912C0B813059F48CE29BE0019616
:1063F0000E94B70E882389F482E080932C0B0DC095
:1064000080912C0B823049F48CE29BE001960E9433
:10641000C90F882311F480932C0B8091380B8823AB
:10642000E1F08091380B813059F488E39BE00196CC
:106430000E94B70E882389F482E08093380B089578
:106440008091380B823049F488E39BE001960E94EA
:10645000C90F882311F48093380B0895CF93DF93ED
:10646000EC0186EA9AE00E94C90F882309F046C031
:106470008091A80A9091A90AAA27BB2788839983AB
:10648000AA83BB83E091AD0AF091AE0A80818D832F
:10649000E091AD0AF091AE0A81818E83E091AD0A60
:1064A000F091AE0A82818F83E091AD0AF091AE0A3D
:1064B00083818887E091AD0AF091AE0A8481898753
:1064C000E091AD0AF091AE0A85818A87E091AD0A2C
:1064D000F091AE0A86818B87E091AD0AF091AE0A09
:1064E00087818C878091AC0A8C8386EA9AE00E942F
:1064F000B70E8823D1F781E090E0BBC281EB9AE030
:106500000E94C90F882309F046C08091B30A909178
:10651000B40AAA27BB2788839983AA83BB83E09107
:10652000B80AF091B90A80818D83E091B80AF091A0
:10653000B90A81818E83E091B80AF091B90A82810B
:106540008F83E091B80AF091B90A83818887E0913E
:10655000B80AF091B90A84818987E091B80AF0916C
:10656000B90A85818A87E091B80AF091B90A8681D3
:106570008B87E091B80AF091B90A87818C87809166
:10658000B70A8C8381EB9AE00E94B70E8823D1F77B
:1065900081E090E06EC28CEB9AE00E94C90F8823E4
:1065A00009F046C08091BE0A9091BF0AAA27BB2776
:1065B00088839983AA83BB83E091C30AF091C40ABC
:1065C00080818D83E091C30AF091C40A81818E831A
:1065D000E091C30AF091C40A82818F83E091C30ADB
:1065E000F091C40A83818887E091C30AF091C40ABC
:1065F00084818987E091C30AF091C40A85818A87E2
:10660000E091C30AF091C40A86818B87E091C30AA6
:10661000F091C40A87818C878091C20A8C838CEBAD
:106620009AE00E94B70E8823D1F781E090E021C262
:1066300087EC9AE00E94C90F882309F046C0809138
:10664000C90A9091CA0AAA27BB2788839983AA837B
:10665000BB83E091CE0AF091CF0A80818D83E091D7
:10666000CE0AF091CF0A81818E83E091CE0AF0911B
:10667000CF0A82818F83E091CE0AF091CF0A838185
:106680008887E091CE0AF091CF0A84818987E091D2
:10669000CE0AF091CF0A85818A87E091CE0AF091E7
:1066A000CF0A86818B87E091CE0AF091CF0A87814D
:1066B0008C878091CD0A8C8387EC9AE00E94B70E7C
:1066C0008823D1F781E090E0D4C182ED9AE00E9466
:1066D000C90F882309F046C08091D40A9091D50A49
:1066E000AA27BB2788839983AA83BB83E091D90A11
:1066F000F091DA0A80818D83E091D90AF091DA0A6B
:1067000081818E83E091D90AF091DA0A82818F83A8
:10671000E091D90AF091DA0A83818887E091D90A59
:10672000F091DA0A84818987E091D90AF091DA0A36
:1067300085818A87E091D90AF091DA0A86818B8770
:10674000E091D90AF091DA0A87818C878091D80A82
:106750008C8382ED9AE00E94B70E8823D1F781E006
:1067600090E087C18DED9AE00E94C90F882309F05F
:1067700046C08091DF0A9091E00AAA27BB27888350
:106780009983AA83BB83E091E40AF091E50A8081B2
:106790008D83E091E40AF091E50A81818E83E09196
:1067A000E40AF091E50A82818F83E091E40AF09196
:1067B000E50A83818887E091E40AF091E50A848103
:1067C0008987E091E40AF091E50A85818A87E09162
:1067D000E40AF091E50A86818B87E091E40AF09162
:1067E000E50A87818C878091E30A8C838DED9AE09E
:1067F0000E94B70E8823D1F781E090E03AC188EE7D
:106800009AE00E94C90F882309F046C08091EA0AE5
:106810009091EB0AAA27BB2788839983AA83BB831D
:10682000E091EF0AF091F00A80818D83E091EF0A08
:10683000F091F00A81818E83E091EF0AF091F00AE5
:1068400082818F83E091EF0AF091F00A838188873B
:10685000E091EF0AF091F00A84818987E091EF0AD4
:10686000F091F00A85818A87E091EF0AF091F00AB1
:1068700086818B87E091EF0AF091F00A87818C87FF
:106880008091EE0A8C8388EE9AE00E94B70E8823EE
:10689000D1F781E090E0EDC083EF9AE00E94C90F4C
:1068A000882309F046C08091F50A9091F60AAA273C
:1068B000BB2788839983AA83BB83E091FA0AF0916E
:1068C000FB0A80818D83E091FA0AF091FB0A8181B5
:1068D0008E83E091FA0AF091FB0A82818F83E09126
:1068E000FA0AF091FB0A83818887E091FA0AF09115
:1068F000FB0A84818987E091FA0AF091FB0A85817D
:106900008A87E091FA0AF091FB0A86818B87E091F1
:10691000FA0AF091FB0A87818C878091F90A8C83AF
:1069200083EF9AE00E94B70E8823D1F781E090E0D0
:10693000A0C08EEF9AE00E94C90F882309F046C0DC
:106940008091000B9091010BAA27BB278883998324
:10695000AA83BB83E091050BF091060B80818D83A8
:10696000E091050BF091060B81818E83E091050B80
:10697000F091060B82818F83E091050BF091060B5D
:1069800083818887E091050BF091060B84818987CC
:10699000E091050BF091060B85818A87E091050B4C
:1069A000F091060B86818B87E091050BF091060B29
:1069B00087818C878091040B8C838EEF9AE00E94F4
:1069C000B70E8823D1F781E090E053C089E09BE0C7
:1069D0000E94C90F882309F046C080910B0B90914B
:1069E0000C0BAA27BB2788839983AA83BB83E091DA
:1069F000100BF091110B80818D83E091100BF091C1
:106A0000110B81818E83E091100BF091110B82812B
:106A10008F83E091100BF091110B83818887E091B7
:106A2000100BF091110B84818987E091100BF0918C
:106A3000110B85818A87E091100BF091110B8681F3
:106A40008B87E091100BF091110B87818C878091DF
:106A50000F0B8C8389E09BE00E94B70E8823D1F74F
:106A600081E090E006C0188219821A821B8280E0C1
:106A700090E0DF91CF910895CF93DF93DC01809177
:106A8000140B882339F484E19BE09093450B8093A9
:106A9000440B21C08091200B882339F480E29BE0D5
:106AA0009093450B8093440B16C080912C0B882348
:106AB00039F48CE29BE09093450B8093440B0BC020
:106AC0008091380B882309F072C088E39BE0909393
:106AD000450B8093440BE091440BF091450B0084EF
:106AE000F185E02DED018D818083E091440BF091E3
:106AF000450B0084F185E02D8E818183E091440B6C
:106B0000F091450B0084F185E02D8F818283E09127
:106B1000440BF091450B0084F185E02D888583833B
:106B2000E091440BF091450B0084F185E02D8985BF
:106B30008483E091440BF091450B0084F185E02DB6
:106B40008A858583E091440BF091450B0084F185A3
:106B5000E02D8B858683E091440BF091450B0084FA
:106B6000F185E02D8C858783E091440BF091450BF6
:106B70008C818783E091440BF091450B8D919C9122
:106B800094838383E091440BF091450B1286E0914E
:106B9000440BF091450B1182E091440BF091450BB1
:106BA0001282E091440BF091450B81E08083DF91EC
:106BB000CF91089589E29AE00E942E32882361F1F4
:106BC00089E29AE00E94820C89E29AE00E942E32C9
:106BD000882311F189E29AE00E94820C89E29AE00E
:106BE0000E942E328823C1F089E29AE00E94820C32
:106BF00089E29AE00E942E32882371F089E29AE0BD
:106C00000E94820C89E29AE00E942E32882321F0B1
:106C100089E29AE00E94820C0895FF920F931F93DD
:106C2000CF93DF93CDB7DEB760970FB6F894DEBF92
:106C30000FBECDBF20E0822F9927880F991F880FA4
:106C4000991F8C010A5B144FF8011082F22EF39405
:106C5000BE016F5F7F4F8F2D0E9457298889F801F1
:106C60008283138211822F2D2B3028F360960FB66A
:106C7000F894DEBF0FBECDBFDF91CF911F910F9172
:106C8000FF900895FC0180819927009719F00197E2
:106C900031F0089582E0838381E0808308958381C9
:106CA000882389F48281882329F481E0818382E02A
:106CB000808308958181813011F4118202C081E0C6
:106CC000818382E080830895FC018081992781304F
:106CD00091059CF0833091051CF0039731F00895E5
:106CE00082E0838383E0808308958381882329F46D
:106CF00080838281882309F48183089520E0822F94
:106D00009927880F991F880F991FFC01EA5BF44FA0
:106D10008381882311F0815083832F5F2B3078F398
:106D2000E6E4FBE0309B04C0CF010E94423603C082
:106D3000CF010E946436EAE4FBE0319904C0CF0140
:106D40000E94423603C0CF010E946436EEE4FBE0AD
:106D5000329904C0CF010E94423603C0CF010E9485
:106D60006436E2E5FBE0499904C0CF010E94423657
:106D700003C0CF010E946436E6E5FBE0349904C00D
:106D8000CF010E94423603C0CF010E946436EAE57B
:106D9000FBE0359904C0CF010E94423603C0CF0109
:106DA0000E946436EEE5FBE0369904C0CF010E94F4
:106DB000423603C0CF010E946436E2E6FBE0379919
:106DC00004C0CF010E94423603C0CF010E94643646
:106DD000E6E6FBE0339904C0CF010E94423603C0CF
:106DE000CF010E946436EAE6FBE04A9904C0CF0175
:106DF0000E94423603C0CF010E946436EEE6FBE0FB
:106E00004B9904C0CF010E9442360895CF010E94E1
:106E1000643608959927853C910509F43FC0863C66
:106E20009105A4F4823C910569F1833C91053CF401
:106E3000803C9105F9F0813C910501F147C0833C0C
:106E40009105C1F1843C910529F140C0813D910536
:106E5000E9F0823D91053CF4863C910519F1873CAF
:106E6000910521F133C0823D910541F1833D9105AA
:106E700049F12CC08091470B9927089580914B0BC5
:106E80009927089580914F0B992708958091530B6E
:106E9000992708958091570B9927089580915B0B4E
:106EA0009927089580915F0B992708958091630B2E
:106EB000992708958091670B9927089580916B0B0E
:106EC0009927089580916F0B992708958EEF90E090
:106ED00008951092B60087E08093B0001092B2003F
:106EE0008EE48093B30082E08093700008950E9446
:106EF00069371092740B1092750B1092760B1092EA
:106F0000770B10927C0B10927D0B0E940D360E9425
:106F1000F8050E94DE240895CF93C82F8091720B4C
:106F2000882311F01092720BA8950E94DA35C230B6
:106F300011F00E94AD31C23009F46FC08091730B23
:106F4000882309F444C08091730B81508093730BA4
:106F50008091740B8F5F8093740B823040F010929D
:106F6000740B0E947E360E9457100E943207809157
:106F7000750B8F5F8093750B843040F01092750B0A
:106F80000E945E100E948F460E94AF438091760B54
:106F90008F5F8093760B8A3030F01092760BC13081
:106FA00011F00E946A0C8091770B8F5F8093770BB2
:106FB000843168F01092770B80917C0B8F5F809307
:106FC0007C0B0E94462C0E94B7100E941B0C8091E3
:106FD0007C0B8A3010F110927C0B8091780B909191
:106FE000790BA0917A0BB0917B0B0196A11DB11D7D
:106FF0008093780B9093790BA0937A0BB0937B0BD3
:107000000E94E62580917D0B8F5F80937D0B8C33F2
:1070100020F010927D0B0E94A525CF9108958091BC
:10702000780B9091790BA0917A0BB0917B0BBC01FE
:10703000CD0108951F920F920FB60F9211248F93D6
:107040001092B20081E08093720B8091730B8F5F7E
:107050008093730B8F910F900FBE0F901F90189518
:107060000E9445420E94FA4360E076E980E090E0A9
:107070000E941544089504C00E948B420E94E94278
:107080000E9475428823C1F70895FC0190E0615089
:107090006F3F21F0819198276150E0F7892F992760
:1070A00008950F931F938C01FC0181818150682FFB
:1070B000C80101960E944538F80180838181992793
:1070C000BC01C8010E94A6421F910F910895AF9282
:1070D000BF92CF92DF92EF92FF920F931F93CF93C5
:1070E000DF93CDB7DEB7C35ED0400FB6F894DEBFF6
:1070F0000FBECDBF6C01FC0181818150682FC6019C
:1071000001960E944538D6019C91981711F00C9475
:10711000D341F6018281882309F0F8C08381992741
:107120008135910509F449C0823591053CF48033DD
:10713000910589F08035910561F1E8C083359105AD
:1071400009F48EC0833591050CF478C0843591051F
:1071500009F4B2C0DBC08E01035D1F4F80E5D8018A
:107160001D928A95E9F785E18EA71FA680E888AB76
:10717000F601848189AB992796012B5F3F4FAC01C3
:10718000B901CE01C2960E945055C8010E945138E3
:10719000BDC08E01035D1F4F80E5D8011D928A9509
:1071A000E9F785E08EA71FA680EA88AB0E946C23D2
:1071B00089ABC8010E945138A9C0F601B4800F2ED6
:1071C000FDE2EF2EFF24F02DEC0EFD1E80E5D70131
:1071D0001D928A95E9F789E18EA71FA681EA88ABFF
:1071E0008E0103581F4FB8018B2D0E949623B9AA18
:1071F0008CE0FE01F296D8010D9001928A95E1F79C
:10720000F801848595859FAF8EAF8685FE01E05C91
:10721000FF4F8083F8018785FE01EF5BFF4F80837E
:107220009927AC01BE0163577F4FCE018E5B9F4F04
:107230000E945055C7010E94513868C00E94242303
:10724000FE01BD9680E5DF011D928A95E9F784E095
:107250008EA71FA682EA88ABCF010E94513856C084
:10726000F601458156818481FE01ED51FF4F8083F7
:10727000813108F04BC080E5FE01BD9611928A95E0
:10728000E9F787E18EA71FA683EA88AB5BAB4AAB21
:10729000FE01ED51FF4F808189ABFE01F4969927E5
:1072A000DA01019724F00E9434560192FACFCE0100
:1072B0008D960E9451382AC0F601458156818481FD
:1072C000FE01ED51FF4F8083813100F5F6013796C5
:1072D0009927DA01019724F001900E944156FACFD4
:1072E000DE019D9680E5FD0111928A95E9F787E020
:1072F0008EA71FA684EA88AB5BAB4AABFE01ED51BB
:10730000FF4F808189ABCD010E945138F601828107
:10731000813011F00C94DC4183819927AA27BB2787
:10732000FC013197E536F10510F00C94C541E65BA0
:10733000FF4FEE0FFF1F0590F491E02D09940E947E
:107340007C21F601B4808B2D8150823210F00C9498
:10735000DC4120E0AE01475F5F4F822F9927DA01C1
:10736000A80FB91FF601E80FF91F82858C932F5FD4
:107370002F3098F3F6018581898386818A838781FE
:107380008B83838D948D9E838D83858D8F83808564
:10739000888781858C83818D888F828D898F6B2DE5
:1073A000CE0101960E94A3286B2DCE0101960E946A
:1073B00097171DA685E08EA711E01FA781E888AB6F
:1073C00019AACE018D960E945138812F0E948C37C8
:1073D0000C94DC41F601B4808B2D8150823208F090
:1073E00046C06B2DCE0101960E94E8288EE18EA743
:1073F00081E08FA782E888ABB9AA89818AAB8A81AC
:107400008BAB8B818CAB8C818EAB8D819E81FE0191
:10741000E85BFF4F918380838F81FE01E65BFF4F26
:10742000808320E0BE016F5F7F4FAE01475F5F4FFB
:10743000822F9927DC01A60FB71FFA01E80FF91F69
:107440008081FD0186AB2F5F2F3090F388858DAB57
:10745000888DFE01EA5BFF4F8083898DFE01E95B29
:10746000FF4F8083CE018D960E945138A5C7FFEF54
:10747000BF1609F0A1C7FE01ED51FF4F1082FE01BA
:10748000ED51FF4F8081982F823208F095C70F2E63
:10749000F3EEEF2EFF24F02DEC0EFD1E6E0108948E
:1074A000C11CD11C8E01075F1F4F892F8F5F682F72
:1074B000CE0101960E94E8288EE18EA781E08FA779
:1074C00082E888ABD7018C918F5F89AB89818AABC9
:1074D0008A818BAB8B818CAB8C818EAB8D819E81B5
:1074E000FE01E85BFF4F918380838F81FE01E65BA5
:1074F000FF4F808320E0822F9927DC01AC0DBD1D5A
:10750000F801E80FF91F8081FD0186AB2F5F2F3056
:1075100090F388858DAB888DFE01EA5BFF4F8083F9
:10752000898DFE01E95BFF4F8083CE018D960E941D
:10753000513881E00E948C37D7018C918F5F8C93FA
:10754000982F823208F4B1CF37C70E947C21F60110
:10755000B480AE0143585F4F96012B5F3F4F8FE0E1
:10756000DA01F90101900D928A95E1F7F60184891B
:10757000FA018787BA018B2D0E943A2981E08FA7F3
:1075800083E888ABB9AA85E08EA7CE018D960E94CC
:10759000513812C7F601B4808B2D81508A3008F51E
:1075A00081E08FA784E888ABB9AA8E0103581F4FEA
:1075B000B8018B2D0E9457298FE0FE01F296D80169
:1075C0000D9001928A95E1F7F8018785FE01EF5B46
:1075D000FF4F808385E18EA7CE018D960E945138A2
:1075E000EBC6FFEFBF1609F0E7C6FE01ED51FF4FF6
:1075F0001082FE01ED51FF4F8081982F8B3008F0F3
:10760000DBC6BB24B3948E0103581F4F0F2EFFE03F
:10761000AF2EF02D0F2EF1E4EF2EFF24F02DEC0E07
:10762000FD1E0F2EF3EECF2EDD24F02DCC0EDD1E31
:10763000BFA684E888AB892F8F5F89ABB8010E9411
:107640005729FE01F296D8012A2D0D9001922A9514
:10765000E1F7F8018785D7018C9385E18EA7CE01EC
:107660008D960E9451388B2D0E948C37F6018081B7
:107670008F5F8083982F8B30D8F29EC60E947C212A
:107680000E94D512A8950E940F16A8950E94FD167B
:10769000A8950E947E0BA8950E945B46A8950E9423
:1076A0004F06A8950E944B2581E08FA786E888ABFE
:1076B00084E08EA7CE018D960E9451387DC684E16C
:1076C0008EA781E08FA787E888AB8DE0A7E4B1E0C3
:1076D000FE01F1960D9001928A95E1F70E940F3814
:1076E0009B01AC01AA27BB278EAFBB27A52F942FE8
:1076F000832F8FAFFE01E05CFF4F2083CE018D967C
:107700000E94513859C60C94000056C6C601049612
:107710000E94312781E08FA789E888AB84E08EA79B
:10772000CE018D960E94513847C681E08FA78AE826
:1077300088AB8CE08EA7CE01C1960E944127CE0176
:107740008D960E94513838C6CE0187960E94D61E6B
:1077500081E08FA781EA88AB8FA189AB88A58AAB2E
:1077600089A58BAB8AA58CAB8BA58DAB8CA58EAB7D
:107770008AE08EA7CE018D960E9451381DC6F60173
:10778000B480F1E2FB15F8F0BE016E5D7F4F8B2DEA
:107790000E94C81F81E08FA782EA88ABB9AA8BA19B
:1077A0008BAB8CA18EAB8AA18AAB8DA19EA1892FB8
:1077B00099278CAB8DA18DAB8AE08EA7CE018D96DB
:1077C0000E945138F9C52FEFB21609F0F5C5FE0138
:1077D000ED51FF4F1082FE01ED51FF4F8081982F38
:1077E000823208F0E9C5FF24F3948F01BE016E5D7B
:1077F0007F4F892F8F5F0E94C81FFFA682EA88AB48
:10780000D8018C918F5F89AB8BA18BAB8CA18EAB98
:107810008AA18AAB8DA19EA1892F99278CAB8DA1BE
:107820008DAB8AE08EA7CE018D960E9451388F2DA8
:107830000E948C37F80180818F5F8083982F82327D
:10784000A8F2BAC5CE014A960E9492208AE08EA77D
:1078500081E08FA780EA88AB88A189AB8E8D8AAB47
:107860008A8D9B8D892F99278BAB8A8D8CAB8D8DC3
:107870008DAB8C8D8EABCE018D960E9451389CC500
:10788000F601648180E00E941B1984E08EA781E0EC
:107890008FA783EA88ABCE018D960E9451388CC5A4
:1078A000DE01A353BF4FF60184818C938581FD01D6
:1078B0008183F6018681FD018283F6018781FD01C6
:1078C0008383F6018085FD018483F6018185FD01B6
:1078D0008583F6018285FD018683F6018385FD019E
:1078E0008783CD010E94231984E08EA781E08FA7B2
:1078F00084EA88ABCE018D960E9451385DC5FE01A9
:10790000E358FF4FA0E0B0E080E190E021E080305C
:10791000920719F40E943C5603C0182E0E943C5650
:10792000F60184819581A681B781FE01EF57FF4F53
:1079300080839183A283B383DE01A358BF4FF601F6
:107940008085FD018087F6018185FD018187F60133
:107950008285FD018287A0E0B0E080E190E021E037
:107960008030920719F40E944D5603C0182E0E94D1
:107970004D5684E08EA781E08FA780EC88ABCE01C6
:107980008D960E94513818C5FE01E358FF4FA0E0C4
:10799000B0E080E190E021E08030920719F40E948D
:1079A0003C5603C0182E0E943C568BE08EA781E007
:1079B0008FA781EC88ABFE01EF57FF4F808191814B
:1079C000A281B38189AB9AABABABBCABFE01E358F0
:1079D000FF4F80858DAB81858EAB82858FABCE01CD
:1079E0008D960E945138E8C48AE38EA781E08FA764
:1079F00080ED88ABFE01F196A8E8B0E082E190E06E
:107A000021E08030920719F40E943C5603C0182EE2
:107A10000E943C56FE01ED5BFF4FAAE9B0E082E117
:107A200090E021E08030920719F40E943C5603C098
:107A3000182E0E943C56FE01EB5AFF4FADEBB0E012
:107A400082E190E021E08030920719F40E943C56D8
:107A500003C0182E0E943C56CE018D960E945138CC
:107A6000ABC484E18EA781E08FA78EED88ABFE01C9
:107A7000F196ACEAB0E080E190E021E0803092073E
:107A800019F40E943C5603C0182E0E943C56CE01A9
:107A90008D960E94513890C40E944B2584E08EA799
:107AA00081E08FA781ED88ABCE018D960E94513881
:107AB00083C488E08EA781E08FA78FED88AB0E94FA
:107AC000DD258BAB0E94E1259AAB89ABFE01ED5120
:107AD000FF4FACEBB0E081E090E021E08030920716
:107AE00019F40E943C5603C0182E0E943C56FE0119
:107AF000ED51FF4F80818CABCE018D960E945138A5
:107B00005BC4FE01E358FF4F80E5DF011D928A95BB
:107B1000E9F7ACEBB0E081E090E021E08030920743
:107B200019F40E944D5603C0182E0E944D56FE01B6
:107B3000E358FF4FA5E8B0E081E090E021E080301D
:107B4000920719F40E944D5603C0182E0E944D56FC
:107B5000FE01E358FF4FA6E8B0E082E090E021E0AC
:107B60008030920719F40E944D5603C0182E0E94CF
:107B70004D5684E08EA781E08FA780EE88ABCE01C2
:107B80008D960E94513818C4DE01AB52BF4FF601EA
:107B900084818C938581FD018183D60116968CE0CA
:107BA000FE01E952FF4F0D9001928A95E1F7FE0127
:107BB000ED51FF4F1082FE01ED51FF4F8081982F54
:107BC0008C30A0F49E012B523F4FDF01F901E90FE9
:107BD000F11D8281882321F08F3F11F08150828333
:107BE0008C918F5F8C93982F8C3080F3CE018B52C9
:107BF0009F4F0E94E32684E08EA781E08FA787EA4B
:107C000088ABCE018D960E945138D6C38E010B529F
:107C10001F4FC8010E94012782E18EA781E08FA734
:107C200088EA88ABD8018C9189ABF80181818AAB55
:107C3000FE01ED51FF4F1082FE01ED51FF4F80819B
:107C4000982F8C3080F49801DF01F901E90FF11DC4
:107C500082818F3F11F08F5F82838C918F5F8C9335
:107C6000982F8C3090F38CE0DE01A952BF4FFE01BB
:107C7000F3960D9001928A95E1F7CE018D960E94C0
:107C800051389AC3F6018481FE01E358FF4F808387
:107C9000D601159680E1FE01E258FF4F0D9001924A
:107CA0008A95E1F7FE01ED51FF4F1082FE01ED5183
:107CB000FF4F8081982F8031A0F49E0123583F4FC1
:107CC000DF01F901E90FF11D8181882321F08F3F48
:107CD00011F0815081838C918F5F8C93982F80312C
:107CE00080F3CE0183589F4F0E94112784E08EA716
:107CF00081E08FA789EA88ABCE018D960E9451382A
:107D00005BC38E0103581F4FC8010E94212785E1E4
:107D10008EA781E08FA78AEA88ABD8018C9189ABC6
:107D2000FE01ED51FF4F1082FE01ED51FF4F8081AA
:107D3000982F803180F49801DF01F901E90FF11DDE
:107D400081818F3F11F08F5F81838C918F5F8C9346
:107D5000982F803190F380E1DE01A258BF4FFE01E1
:107D6000F2960D9001928A95E1F7CE018D960E94D0
:107D7000513822C3F601B48085819927982F88272E
:107D80002681820F911DBC018B2D0E94FF2085E072
:107D90008EA781E08FA782EC88ABB9AACE018D9621
:107DA0000E94513809C3F601B4808CE08EA781E0AF
:107DB0008FA783EC88ABB9AA8B2D0E94BD208AAB1C
:107DC0008B2D0E94D920892F99278BAB8B2D0E9458
:107DD000D9208CAB8B2D0E942821892F99278DAB20
:107DE0008B2D0E9428218EAB8B2D0E944021892F44
:107DF00099278FAB8B2D0E94402188AFCE018D96A5
:107E00000E945138D9C220E0F601848181FD21E031
:107E1000F601848182FD2260F6018181863029F499
:107E20006581822F0E945821C7C260E0822F0E9484
:107E30005821C2C20E945D2184E08EA781E08FA7F5
:107E400085EC88ABCE018D960E945138B5C2F60103
:107E5000B4809E0123583F4F9581492F4170D9012D
:107E60008C91887F9670842B892B8C938681978147
:107E7000F90192838183F60180859185F9019483CC
:107E80008383F6018685F9018187F6018785F901EB
:107E90008287F60182859385F90196838583F601B1
:107EA00084859585F90190878783F6018089F9019A
:107EB0008387F6018189F9018487F6018289F901B6
:107EC0008587F6018389F9018687D60154968FE06C
:107ED000FE01E457FF4F0D9001928A95E1F7F601FC
:107EE00083A1F901868FF60184A1F901878FF6013C
:107EF00085A1F90180A3F60186A1F90181A315E00E
:107F0000D6019796FE01E156FF4F812F0D90019209
:107F10008A95E1F7F60184A595A5A6A5B7A5F9016F
:107F200087A390A7A1A7B2A7F60180A9F90183A70B
:107F3000B9018B2D0E94C32781E08FA782ED88AB0A
:107F40001EA7B9AACE018D960E94513835C2F601FE
:107F5000B4808E0103581F4FB8018B2D0E94FB2760
:107F600081E08FA783ED88AB81E38EA7B9AAD80102
:107F70009C91292F21708AA9887F9670822B892B4A
:107F80008AABF801818192819CAB8BAB8381948118
:107F90009EAB8DAB81858BAF82858CAF85819681C1
:107FA00098AF8FAB878190859AAF89AF83858DAF6E
:107FB00084858EAF85858FAF8685FE01E05CFF4F9F
:107FC00080838FE0DE01A457BF4FFE01EF5BFF4FC0
:107FD0000D9001928A95E1F7F801868DFE01E05B34
:107FE000FF4F8083F801878DFE01EF5AFF4F80839A
:107FF000F80180A1FE01EE5AFF4F8083F80181A1B4
:10800000FE01ED5AFF4F808385E0DE01A156BF4F90
:10801000FE01EC5AFF4F0D9001928A95E1F7F801AD
:1080200087A190A5A1A5B2A5FE01E75AFF4F8083C5
:108030009183A283B383F80183A5FE01E35AFF4F26
:108040008083CE018D960E945138B6C1F601B4806E
:10805000AE0143585F4F828DDA018C93838DFA0114
:108060008183F601848DFA018283F6018681FA010B
:108070008383F6018781FA018483F6018085FA0102
:108080008583F6018185FA018683F6018285FA01EE
:108090008783F601858DFA01878BC6010B962FE049
:1080A000FE01EB57FF4FDC010D9001922A95E1F79D
:1080B000BA018B2D0E94332881E08FA784ED88AB15
:1080C00085E08EA7B9AACE018D960E94513874C161
:1080D000F601B4808E0103581F4FB8018B2D0E940A
:1080E0006B2881E08FA785ED88AB8FE18EA7B9AAB9
:1080F000D8018C91FE01E95BFF4F8083F8018181FB
:10810000FE01E85BFF4F8083F8018281FE01E75B9F
:10811000FF4F8083F80183818BAB84818CAB858199
:108120008DAB86818EAB87818FAB8789FE01E65B45
:10813000FF4F80838FE0DE01AB57BF4FFE01F89603
:108140000D9001928A95E1F7CE018D960E945138EB
:1081500033C1F6013496A0E0B9E080E190E021E07F
:108160008030920719F40E944D5603C0182E0E94C9
:108170004D5681E08FA783EE88AB84E08EA7CE01B9
:108180008D960E94513818C181E08FA784EE88AB8C
:1081900084E18EA7FE01F196A0E0B9E080E190E0D5
:1081A00021E08030920719F40E943C5603C0182E3B
:1081B0000E943C56CE018D960E945138FDC0F601BA
:1081C000B480C6010596BC018B2D0E94512781E029
:1081D0008FA788ED88AB85E08EA7B9AACE018D96D2
:1081E0000E945138E9C0F601B48081E08FA789ED83
:1081F00088AB8DE18EA7B9AABE016E5C7F4F8B2D37
:108200000E948A27CE018D960E945138D5C0C601A2
:1082100005960E94C52981E08FA786ED88AB85E091
:108220008EA7CE018D960E945138C6C081E08FA7DF
:1082300087ED88AB8DE18EA7CE01C2960E94D5292D
:10824000CE018D960E945138B7C0F601B480C601A8
:1082500004960E94E52981E08FA78AED88AB85E02E
:108260008EA7B9AACE018D960E945138A5C0F601FD
:10827000B48081E08FA78BED88AB8AE48EA7BE0126
:108280006F5C7F4F8B2D0E94122ACE018D960E942B
:10829000513892C0F601B4808B2D0E94EA0B81E028
:1082A0008FA78CED88ABB9AA85E08EA7CE018D96FD
:1082B0000E94513881C0F6014481558181E08FA729
:1082C0008DED88AB86E18EA75AAB49ABFE01ED512F
:1082D000FF4F1082FE01ED51FF4F8081982F8031BA
:1082E000C8F48E010F5F1F4FBF01892F99279C0192
:1082F000200F311F840F951FAA27BB27ABBFFC019E
:108300008791F90182ABDB018C918F5F8C93982F61
:10831000803158F3CE018D960E9451384DC0F60140
:108320003496A2E8BFE080E190E021E0803092073F
:1083300019F40E944D5603C0182E0E944D5681E03C
:108340008FA781EE88AB84E08EA7CE018D960E9428
:10835000513832C081E08FA782EE88AB84E18EA7CE
:10836000FE01F196A2E8BFE080E190E021E08030DC
:10837000920719F40E943C5603C0182E0E943C56E6
:10838000CE018D960E94513817C081E08FA780E8FA
:1083900088AB85E08EA7F601838189ABCE018D96EF
:1083A0000E94513809C085E08EA71FA681E088ABE6
:1083B000CE018D960E945138CD51DF4F0FB6F89403
:1083C000DEBF0FBECDBFDF91CF911F910F91FF9008
:1083D000EF90DF90CF90BF90AF900895CF93DF9351
:1083E000CDB7DEB72A970FB6F894DEBF0FBECDBF6C
:1083F00081E08B8388E88C8384E08A83CE010196B8
:108400000E9451382A960FB6F894DEBF0FBECDBF3A
:10841000DF91CF9108950F931F93CF93DF93CDB743
:10842000DEB7C055D0400FB6F894DEBF0FBECDBF4B
:108430008A0121E02B832DE52C839E838D836F831E
:1084400020E0261780F4AE01485F5F4F822F992706
:10845000DA01A80FB91FF801E80FF91F80818C938A
:108460002F5F261798F38FE08A83CE0101960E9432
:108470005138C05BDF4F0FB6F894DEBF0FBECDBFE3
:10848000DF91CF911F910F91089548EC50E060E08B
:1084900070E08FE79BE00E945D551092470C1092B0
:1084A000480C10927E0B0895382F2091480C8FE7CE
:1084B0009BE0FC01E20FF11D30838091480C8F5F3F
:1084C0008093480C80917E0B8F5F80937E0B809110
:1084D0007E0B883C18F00E94454208958091480C1C
:1084E000883C10F01092480C08959091480C8091AF
:1084F000470C981738F08091480C9091470C891BD5
:10850000992708959091480C8091470C981B892FCA
:108510008853992708952091470C8FE79BE0FC0131
:10852000E20FF11DE0818091470C8F5F8093470C33
:1085300080917E0B815080937E0B8091470C883C0C
:1085400010F01092470C8E2F992708950F931F93C8
:10855000CF93DF938C01EB0180EC0E943B44219789
:108560008FEFCF3FD80769F1CE0165E070E00E9440
:10857000AD55892B19F081E00E948C37F80180817C
:108580009927803C910521F08B3D910541F00EC06B
:108590008BED0E943B448CED0E943B440BC08BED65
:1085A0000E943B448DED0E943B4404C0F801808151
:1085B0000E943B440F5F1F4F2197FFEFCF3FDF0724
:1085C00099F680EC0E943B44DF91CF911F910F916F
:1085D00008950F931F93382F8091490C9927009786
:1085E00019F00197C1F059C0303C09F056C0109203
:1085F0004A0C20914A0C8CE49CE0FC01E20FF11D36
:1086000030832F5F20934A0C81E08093490C84E6ED
:1086100080934B0C42C0303C99F580914A0C8230DB
:10862000F0F080914A0C0CE41CE0F801E80FF11D19
:1086300030838F5F80934A0C82E08093490C1092C4
:108640004B0CA80160914A0CC8010E945843C80114
:108650000E9467381092490C10924A0C1EC010926A
:108660004A0C20914A0C8CE49CE0FC01E20FF11DC5
:1086700030832F5F20934A0C84E680934B0C0DC00F
:1086800020914A0C8CE49CE0FC01E20FF11D308348
:1086900080914A0C8F5F80934A0C80914A0C8936F6
:1086A00020F01092490C10924A0C1F910F910895DE
:1086B000FC01DA0161506F3FF1F02081822F992790
:1086C000803C910521F08B3D910519F010C0319649
:1086D00010C031962081822F99278C3D910521F081
:1086E0008D3D910519F003C020EC01C02BED2D93B9
:1086F0003196615010F7089580914B0C882389F0D2
:1087000080914B0C815080934B0C90914B0C992392
:1087100041F48091490C813021F490934A0C90935C
:10872000490C089585B1807F85B984B1876084B98B
:1087300081E58CBD81E08DBD08958EBD0DB407FE31
:10874000FDCF8EB5992708950E94F8439C9AA4986E
:108750008FE08093B60CA4986A9862980895CF939E
:10876000DF93CDB7DEB728970FB6F894DEBF0FBE04
:10877000CDBFA49B11C062990DC08091B50C85300E
:1087800018F0A4980E9411188091B50C8F5F809307
:10879000B50C02C01092B50CCE0101960E94922039
:1087A00029813A8181E590E0289FA001299F500D01
:1087B000389F500D1124CA01880F892F881F990BEB
:1087C00091950E94F9438D81882319F48F81882324
:1087D00011F0A49A01C0A49828960FB6F894DEBFB1
:1087E0000FBECDBFDF91CF9108958093B60C089551
:1087F000089508951092B80C1092B70C86E08093FB
:10880000C20088E98093C10060E875E280E090E0F2
:108810000E94154481E08093570F1092580F0895DD
:108820009093B80C8093B70C08959B01AC01DC01C8
:10883000CB01689412F8880F991FAA1FBB1F1694CA
:10884000D1F780509C4DAB40BF4F689413F8220F76
:10885000331F441F551F1694D1F7BC01CD010E9450
:10886000C055DA01C9010197292F33272093C5008C
:108870008093C4000895982F8091C00085FFFCCF9D
:108880009093C60008950F931F93CF93DF938C01AD
:10889000EB0121978FEFCF3FD80751F0F80181917D
:1088A0008F010E943B442197FFEFCF3FDF07B1F7D5
:1088B00081E090E0DF91CF911F910F9108951F9279
:1088C0000F920FB60F9211242F933F934F935F9304
:1088D0006F937F938F939F93AF93BF93EF93FF9388
:1088E0008091C6000E945442FF91EF91BF91AF91D9
:1088F0009F918F917F916F915F914F913F912F91B8
:108900000F900FBE0F901F901895DC01FB01415096
:1089100050408FEF4F3F580741F081918D93415068
:1089200050408FEF4F3F5807C1F70895DC01FB011E
:10893000415050408FEF4F3F580769F091918D9112
:10894000891719F081E090E00895415050408FEF71
:108950004F3F580799F780E090E00895CF93DF9359
:10896000DC01FB0160E0462F91E0562F80818032D0
:1089700031F4692F9F5F319680818032D1F38081FD
:10898000882379F08081803219F4442309F4492F37
:108990008081803209F040E09F5F3196808188239A
:1089A00089F7442331F48081882311F4492F01C0D1
:1089B000462F262F3327E901C91BD109EC0FFD1FD4
:1089C0003196842F9927821B930B0197181619064D
:1089D00024F4942F961B915001C090E091509F3F3A
:1089E00029F081918D935F5F9150D8F71C925F5F62
:1089F000852F9927DF91CF910895FC0190E0819117
:108A0000882331F09F5F8191882311F09F3FD1F738
:108A1000892F99270895DC01FB018081882329F0A3
:108A200081918D9380818823D9F71C9208950F93AB
:108A30001F93CF93DF93082F162FFA0141E0C0E177
:108A4000D7E2C901BE010E94AD556115710581F0E3
:108A50006C9FC0016D9F900D7C9F900D1124281B71
:108A6000390B862F805D8193440F01E015E00AC029
:108A7000153040F0002319F080E3819302C080E2BA
:108A800081934F5FC8EED3E0C901BE010E94AD558E
:108A90006115710581F06C9FC0016D9F900D7C9FE9
:108AA000900D1124281B390B862F805D81934F5F19
:108AB00001E014E00AC0143040F0002319F080E314
:108AC000819302C080E281934F5FC4E6D0E0C90188
:108AD000BE010E94AD556115710581F04F5F6C9F1D
:108AE000C0016D9F900D7C9F900D1124281B390BA8
:108AF000862F805D819301E013E00AC0133040F0BF
:108B00004F5F002319F080E3819302C080E28193DC
:108B1000C9016AE070E00E94AD556115710591F0E0
:108B20004F5FCB01880F991F880F991F880F991FDE
:108B3000860F971F860F971F281B390B862F805D86
:108B400081930AC0123040F04F5F002319F080E398
:108B5000819302C080E28193822F805D8193108295
:108B6000842F9927DF91CF911F910F910895FC01D8
:108B7000262F862F82958F708A3038F06AE00E9407
:108B80008D55892F8F5B819309C0862F82958F70B9
:108B90006AE00E948D55892F805D8193822F8F70AE
:108BA0008A3038F06AE00E948D55892F8F5B808370
:108BB0000895822F8F706AE00E948D55892F805D05
:108BC00080830895EF92FF920F931F937C018B0196
:108BD000872F9927682FC7010E94B745C801907059
:108BE000682FC7010E94B7451F910F91FF90EF902A
:108BF0000895CF92DF92EF92FF920F931F936C0133
:108C00007A018B01CB01AA27BB27BC01C6010E94B8
:108C1000E245D801C701A070B070BC01C6010E9436
:108C2000E2451F910F91FF90EF90DF90CF90089554
:108C30001F93CF93DF93CDB7DEB768970FB6F89445
:108C4000DEBF0FBECDBF10E0BE016F5F7F4F812F33
:108C50000E946B28212F3327C901880F991F880F85
:108C6000991F880F991F820F931FFC01E754F34F40
:108C7000898185838A8186838B8187838C818083A8
:108C80008D8181838E8182838F8183838885848394
:108C9000888D8087F901E951F24F10821F5F1431EE
:108CA00098F268960FB6F894DEBF0FBECDBFDF9185
:108CB000CF911F9108951F93CF93DF93CDB7DEB768
:108CC00068970FB6F894DEBF0FBECDBF10E0A89531
:108CD00019821A821B821C821D821E821F821886A4
:108CE000188E8FE0189FC00111248459994FBC0140
:108CF000CE0109960E943C55BE016F5F7F4F812FC8
:108D00000E9433281F5F143110F368960FB6F89451
:108D1000DEBF0FBECDBFDF91CF911F910895CF93DE
:108D2000C0E086E0C89FC0011124FC01E159F24F68
:108D3000F0936E0DE0936D0D80819181009719F095
:108D4000019791838083E0916D0DF0916E0D82818A
:108D50009381009719F0019793838283E0916D0DC1
:108D6000F0916E0D84819581009719F0019795839C
:108D700084832C2F3327C901880F991F880F991FCF
:108D8000880F991F820F931FFC01E754F34F8081D6
:108D9000882319F48181882321F08C2F8F5D0E9414
:108DA000E047CF5FC43108F4BCCFCF910895992735
:108DB0008730910509F466C088309105ACF48430A1
:108DC000910509F43EC08530910534F48230910557
:108DD00011F1039759F198C08530910509F43CC011
:108DE000069709F444C090C08A30910509F46BC01D
:108DF0008B30910544F48830910509F44EC00997F1
:108E000009F456C081C08B30910509F467C00C97F6
:108E100009F46FC079C080EC0E940A37882319F0EA
:108E200081E090E0089580E090E0089581EC0E9458
:108E30000A37882319F081E090E0089580E090E0FF
:108E4000089582EC0E940A37882319F081E090E0AF
:108E5000089580E090E0089581ED0E940A3788230C
:108E600019F081E090E0089580E090E0089584ECAE
:108E70000E940A37882319F081E090E0089580E08D
:108E800090E0089585EC0E940A37882319F081E06C
:108E900090E0089580E090E0089586EC0E940A3703
:108EA000882319F081E090E0089580E090E0089533
:108EB00087EC0E940A37882319F081E090E008953A
:108EC00080E090E0089583EC0E940A37882319F02F
:108ED00081E090E0089580E090E0089582ED0E94A6
:108EE0000A37882319F081E090E0089580E090E04F
:108EF000089583ED0E940A37882319F081E090E0FD
:108F0000089580E090E0089580E090E008950F9348
:108F1000CF93DF93CDB7DEB721970FB6F894DEBFBE
:108F20000FBECDBF89838150843170F000E021E015
:108F3000AE014F5F5F4F69E071E08EE591E00E9406
:108F4000C62380E090E007C089819927FC01EA519F
:108F5000F24F8081992721960FB6F894DEBF0FBE9D
:108F6000CDBFDF91CF910F9108950F93CF93DF93F2
:108F7000CDB7DEB721970FB6F894DEBF0FBECDBFD9
:108F80008983843160F000E021E0AE014F5F5F4FE4
:108F900064E171E08EE591E00E94C62307C08981FB
:108FA00027EE3DE0F901E80FF11D608321960FB631
:108FB000F894DEBF0FBECDBFDF91CF910F91089522
:108FC000DF92EF92FF920F931F93CF93DF93CDB772
:108FD000DEB721970FB6F894DEBF0FBECDBF198262
:108FE000813209F46DC0823219F481E0898368C04E
:108FF000833219F482E0898363C0843219F483E0F8
:1090000089835EC0853219F484E0898359C0863231
:1090100019F485E0898354C0873219F486E0898386
:109020004FC0883219F487E089834AC0893219F425
:1090300088E0898345C08A3219F489E0898340C079
:109040008B3219F48AE089833BC08C3219F48BE0AF
:10905000898336C08D3219F48CE0898331C08E3219
:1090600019F48DE089832CC08F3219F48EE0898346
:1090700027C0803319F48FE0898322C0813319F42B
:1090800080E189831DC0823319F481E1898318C08E
:10909000833319F482E1898313C0843319F483E1A3
:1090A00089830EC000E021E0AE014F5F5F4F69E4AD
:1090B00071E08EE591E00E94C62380E090E05EC7FB
:1090C000FF24EF2CDF2C298186E0289FC00111248A
:1090D0008159924F90936E0D80936D0D3327C90186
:1090E000880F991F880F991F880F991F820F931F50
:1090F000FC01E754F34F8081882309F4A0C18981E2
:10910000282F3327C901880F991F880F991F880FAF
:10911000991F820F931FFC01E754F34F80818F3F0B
:1091200019F4EE24E3948BC18981282F332709EBAE
:109130001CE0C901880F991F880F991F880F991F7C
:10914000820F931FFC01E00FF11FE0818E2F8250F0
:109150008B3008F04CC08E2F0E94D746482F898153
:10916000282F3327C901880F991F880F991F880F4F
:10917000991F820F931FFC01E00FF11F808580FF74
:1091800002C081E04827442369F0E0916D0DF09121
:109190006E0D80819181892B19F4EE24E3944FC1E7
:1091A000EE244DC1A0916D0DB0916E0D8981282FD7
:1091B0003327C901880F991F880F991F880F991F9E
:1091C000820F931FFC01E754F34F958185E0989F30
:1091D000C00111248D939C93E0916D0DF0916E0D63
:1091E00080819181019691838083EE2428C18981B9
:1091F000282F332709EB1CE0C901880F991F880F1E
:10920000991F880F991F820F931FFC01E00FF11F18
:10921000E0818E2F8D50803208F04CC08F5F0E940D
:10922000ED0B482F8981282F3327C901880F991FFB
:10923000880F991F880F991F820F931FFC01E00F61
:10924000F11F808580FF02C081E04827442369F038
:10925000E0916D0DF0916E0D80819181892B19F453
:10926000EE24E394ECC0EE24EAC0A0916D0DB09121
:109270006E0D8981282F3327C901880F991F880F08
:10928000991F880F991F820F931FFC01E754F34F1A
:10929000958185E0989FC00111248D939C93E09166
:1092A0006D0DF0916E0D8081918101969183808387
:1092B000EE24C5C08981282F332709EB1CE0C901A2
:1092C000880F991F880F991F880F991F820F931F6E
:1092D000FC01E00FF11FE0818E2F8D52823208F0E9
:1092E0004CC08F5F0E944C20482F8981282F332744
:1092F000C901880F991F880F991F880F991F820F26
:10930000931FFC01E00FF11F808580FF02C081E008
:109310004827442369F0E0916D0DF0916E0D808136
:109320009181892B19F4EE24E39489C0EE2487C03F
:10933000A0916D0DB0916E0D8981282F3327C90141
:10934000880F991F880F991F880F991F820F931FED
:10935000FC01E754F34F958185E0989FC0011124EB
:109360008D939C93E0916D0DF0916E0D80819181B4
:10937000019691838083EE2462C08981282F332750
:1093800009EB1CE0C901880F991F880F991F880FEE
:10939000991F820F931FFC01E00FF11FE0818E2FB8
:1093A0008F548F3008F04BC08F5F0E948747482F43
:1093B0008981282F3327C901880F991F880F991F8A
:1093C000880F991F820F931FFC01E00FF11F80850A
:1093D00080FF02C081E04827442369F0E0916D0DD1
:1093E000F0916E0D80819181892B19F4EE24E39424
:1093F00026C0EE2424C0A0916D0DB0916E0D898120
:10940000282F3327C901880F991F880F991F880FAC
:10941000991F820F931FFC01E754F34F958185E05C
:10942000989FC00111248D939C93E0916D0DF09154
:109430006E0D80819181019691838083EE248981D4
:10944000282F3327C901880F991F880F991F880F6C
:10945000991F820F931FFC01E754F34F81818823EA
:1094600011F4F82EA4C18981282F3327C901880F50
:10947000991F880F991F880F991F820F931FFC0156
:10948000E754F34F81818F3F19F4FF24F3948FC188
:109490008981282F332709EB1CE0C901880F991F08
:1094A000880F991F880F991F820F931FFC01E00FEF
:1094B000F11F9181892F82508B3008F04DC0892F88
:1094C0000E94D746482F8981282F3327C901880F4A
:1094D000991F880F991F880F991F820F931FFC01F6
:1094E000E00FF11F808581FF02C081E048274423FF
:1094F00069F0E0916D0DF0916E0D82819381892B61
:1095000019F4FF24F39453C1FF2451C1A0916D0DB0
:10951000B0916E0D8981282F3327C901880F991FBB
:10952000880F991F880F991F820F931FFC01E75422
:10953000F34F968185E0989FC0011124FD0193832C
:109540008283E0916D0DF0916E0D82819381019681
:1095500093838283FF242BC18981282F332709EB32
:109560001CE0C901880F991F880F991F880F991F48
:10957000820F931FFC01E00FF11F9181892F8D5005
:10958000803208F04DC08F5F0E94ED0B482F89811B
:10959000282F3327C901880F991F880F991F880F1B
:1095A000991F820F931FFC01E00FF11F808581FF3F
:1095B00002C081E04827442369F0E0916D0DF091ED
:1095C0006E0D82819381892B19F4FF24F394EFC0EF
:1095D000FF24EDC0A0916D0DB0916E0D8981282FF3
:1095E0003327C901880F991F880F991F880F991F6A
:1095F000820F931FFC01E754F34F968185E0989FFB
:10960000C0011124FD0193838283E0916D0DF091DF
:109610006E0D82819381019693838283FF24C7C05C
:109620008981282F332709EB1CE0C901880F991F76
:10963000880F991F880F991F820F931FFC01E00F5D
:10964000F11F9181892F8D52823208F04DC08F5FBA
:109650000E944C20482F8981282F3327C901880F69
:10966000991F880F991F880F991F820F931FFC0164
:10967000E00FF11F808581FF02C081E0482744236D
:1096800069F0E0916D0DF0916E0D82819381892BCF
:1096900019F4FF24F3948BC0FF2489C0A0916D0DB1
:1096A000B0916E0D8981282F3327C901880F991F2A
:1096B000880F991F880F991F820F931FFC01E75491
:1096C000F34F968185E0989FC0011124FD0193839B
:1096D0008283E0916D0DF0916E0D828193810196F0
:1096E00093838283FF2463C08981282F332709EB6A
:1096F0001CE0C901880F991F880F991F880F991FB7
:10970000820F931FFC01E00FF11F9181892F8F546D
:109710008F3008F04CC08F5F0E948747482F8981A7
:10972000282F3327C901880F991F880F991F880F89
:10973000991F820F931FFC01E00FF11F808581FFAD
:1097400002C081E04827442369F0E0916D0DF0915B
:109750006E0D82819381892B19F4FF24F39427C025
:10976000FF2425C0A0916D0DB0916E0D8981282F29
:109770003327C901880F991F880F991F880F991FD8
:10978000820F931FFC01E754F34F968185E0989F69
:10979000C0011124FD0193838283E0916D0DF0914E
:1097A0006E0D82819381019693838283FF24898148
:1097B000282F3327C901880F991F880F991F880FF9
:1097C000991F820F931FFC01E754F34F8281882376
:1097D00011F4D82EA4C18981282F3327C901880FFD
:1097E000991F880F991F880F991F820F931FFC01E3
:1097F000E754F34F82818F3F19F4DD24D3948FC156
:109800008981282F332709EB1CE0C901880F991F94
:10981000880F991F880F991F820F931FFC01E00F7B
:10982000F11F9281892F82508B3008F04DC0892F13
:109830000E94D746482F8981282F3327C901880FD6
:10984000991F880F991F880F991F820F931FFC0182
:10985000E00FF11F808582FF02C081E0482744238A
:1098600069F0E0916D0DF0916E0D84819581892BE9
:1098700019F4DD24D39453C1DD2451C1A0916D0DA1
:10988000B0916E0D8981282F3327C901880F991F48
:10989000880F991F880F991F820F931FFC01E754AF
:1098A000F34F978185E0989FC0011124FD019583B6
:1098B0008483E0916D0DF0916E0D84819581019608
:1098C00095838483DD242BC18981282F332709EBDD
:1098D0001CE0C901880F991F880F991F880F991FD5
:1098E000820F931FFC01E00FF11F9281892F8D5091
:1098F000803208F04DC08F5F0E94ED0B482F8981A8
:10990000282F3327C901880F991F880F991F880FA7
:10991000991F820F931FFC01E00FF11F808582FFCA
:1099200002C081E04827442369F0E0916D0DF09179
:109930006E0D84819581892B19F4DD24D394EFC0B9
:10994000DD24EDC0A0916D0DB0916E0D8981282FA1
:109950003327C901880F991F880F991F880F991FF6
:10996000820F931FFC01E754F34F978185E0989F86
:10997000C0011124FD0195838483E0916D0DF09168
:109980006E0D84819581019695838483DD24C7C003
:109990008981282F332709EB1CE0C901880F991F03
:1099A000880F991F880F991F820F931FFC01E00FEA
:1099B000F11F9281892F8D52823208F04DC08F5F46
:1099C0000E944C20482F8981282F3327C901880FF6
:1099D000991F880F991F880F991F820F931FFC01F1
:1099E000E00FF11F808582FF02C081E048274423F9
:1099F00069F0E0916D0DF0916E0D84819581892B58
:109A000019F4DD24D3948BC0DD2489C0A0916D0DA1
:109A1000B0916E0D8981282F3327C901880F991FB6
:109A2000880F991F880F991F820F931FFC01E7541D
:109A3000F34F978185E0989FC0011124FD01958324
:109A40008483E0916D0DF0916E0D84819581019676
:109A500095838483DD2463C08981282F332709EB14
:109A60001CE0C901880F991F880F991F880F991F43
:109A7000820F931FFC01E00FF11F9281892F8F54F9
:109A80008F3008F04CC08F5F0E948747482F898134
:109A9000282F3327C901880F991F880F991F880F16
:109AA000991F820F931FFC01E00FF11F808582FF39
:109AB00002C081E04827442369F0E0916D0DF091E8
:109AC0006E0D84819581892B19F4DD24D39427C0F0
:109AD000DD2425C0A0916D0DB0916E0D8981282FD8
:109AE0003327C901880F991F880F991F880F991F65
:109AF000820F931FFC01E754F34F978185E0989FF5
:109B0000C0011124FD0195838483E0916D0DF091D6
:109B10006E0D84819581019695838483DD2449812E
:109B2000842F99279C01220F331F220F331F220FEE
:109B3000331F280F391FF901E754F34F8081882321
:109B400009F45AC18181882309F456C1828188238E
:109B500009F452C18381882309F077C0EE20C9F14E
:109B6000FF20B9F18481882361F46D2D842F0E9438
:109B7000B547DD2019F081E090E000C280E090E080
:109B8000FDC18981282F3327C901880F991F880FAC
:109B9000991F880F991F820F931FFC01E754F34F01
:109BA0008481823079F460E0ED1409F461E0898108
:109BB0000E94B547ED1419F481E090E0DFC180E028
:109BC00090E0DCC161E089810E94B54781E090E0CE
:109BD000D5C14981242F3327C901880F991F880FC8
:109BE000991F880F991F820F931FFC01E754F34FB1
:109BF0008481823049F4DD2039F461E0842F0E94B1
:109C0000B54781E090E0BAC14981842F99279C0132
:109C1000220F331F220F331F220F331F280F391F2C
:109C2000F901E754F34F6481613041F4DD2031F0F4
:109C3000842F0E94B54781E090E0A0C160E0898157
:109C40000E94B54780E090E099C14981842F99270F
:109C50009C01220F331F220F331F220F331F280FA7
:109C6000391FF901E754F34F8381823009F040C076
:109C7000EF14B9F58481882361F46D2D842F0E943F
:109C8000B547DD2019F081E090E078C180E090E0F8
:109C900075C18981282F3327C901880F991F880F23
:109CA000991F880F991F820F931FFC01E754F34FF0
:109CB0008481823079F460E0ED1409F461E08981F7
:109CC0000E94B547ED1419F481E090E057C180E09F
:109CD00090E054C161E089810E94B54781E090E045
:109CE0004DC160E089810E94B54780E090E046C1A7
:109CF000EE2019F4FF2009F443C04981242F3327B3
:109D0000C901880F991F880F991F880F991F820F0B
:109D1000931FFC01E754F34F8481882361F46D2D78
:109D2000842F0E94B547DD2019F081E090E026C124
:109D300080E090E023C14981242F3327C901880F97
:109D4000991F880F991F880F991F820F931FFC017D
:109D5000E754F34F8481823061F46D2D842F0E948B
:109D6000B547DD2019F081E090E008C180E090E087
:109D700005C161E089810E94B54781E090E0FEC0A5
:109D80004981842F99279C01220F331F220F331FF3
:109D9000220F331F280F391FF901E754F34F648155
:109DA000613041F4DD2009F1842F0E94B54781E044
:109DB00090E0E4C04981242F3327C901880F991FFF
:109DC000880F991F880F991F820F931FFC01E7547A
:109DD000F34F8481823049F4DD2039F461E0842F2F
:109DE0000E94B54781E090E0C9C060E089810E948F
:109DF000B54780E090E0C2C04981842F99279C013B
:109E0000220F331F220F331F220F331F280F391F3A
:109E1000F901E754F34F8081882309F44DC0818113
:109E2000882309F449C08381882391F4EE2049F006
:109E3000FF2039F061E0842F0E94B54781E090E077
:109E40009DC060E089810E94B54780E090E096C0A7
:109E50004981242F3327C901880F991F880F991F23
:109E6000880F991F820F931FFC01E754F34F8381E2
:109E7000823081F4EF1439F461E0842F0E94B547F9
:109E800081E090E07BC060E089810E94B54780E07E
:109E900090E074C0EE2011F4FF2039F061E0898178
:109EA0000E94B54781E090E069C060E089810E942E
:109EB000B54780E090E062C04981842F99279C01DA
:109EC000220F331F220F331F220F331F280F391F7A
:109ED000F901E754F34F8181882309F44DC0828151
:109EE000882309F449C08481882391F4EE2049F045
:109EF000FF2039F061E0842F0E94B54781E090E0B7
:109F00003DC060E089810E94B54780E090E036C0A6
:109F10004981242F3327C901880F991F880F991F62
:109F2000880F991F820F931FFC01E754F34F848120
:109F3000823081F4EF1439F461E0842F0E94B54738
:109F400081E090E01BC060E089810E94B54780E01D
:109F500090E014C0EE2011F4FF2039F061E0898117
:109F60000E94B54781E090E009C060E089810E94CD
:109F7000B54780E090E002C080E090E021960FB607
:109F8000F894DEBF0FBECDBFDF91CF911F910F912F
:109F9000FF90EF90DF900895CF93DF93CDB7DEB7BA
:109FA00021970FB6F894DEBF0FBECDBF282F04B6A1
:109FB00003FE28C0FE013196ACEBB0E081E090E0FA
:109FC00031E08030930719F40E943C5603C0182EEC
:109FD0000E943C568981843190F48F5F8983FE0111
:109FE0003196ACEBB0E081E090E031E08030930757
:109FF00019F40E944D5603C0182E0E944D5684B786
:10A00000877F84BF80916000886180936000209387
:10A0100060008091600088608093600021960FB698
:10A02000F894DEBF0FBECDBFDF91CF910895EF92C0
:10A03000FF920F931F937B018C0120E030E040E002
:10A040005FE40E947B5288239CF020E030E040E0F7
:10A050005FECC801B7010E946551DC01CB01BC0176
:10A06000CD010E941553605070408040904804C05C
:10A07000C801B7010E9415531F910F91FF90EF90F7
:10A080000895A0E0B0E0E7E4F0E50C94FD558C0104
:10A090007B015A01DC018C91823058F0FB019081E8
:10A0A000923010F4A7010BC1843029F4943009F4E4
:10A0B000A6C0A80104C19430A9F3923009F4A9C044
:10A0C000823081F3F801C280D380FB016281738109
:10A0D000F8012481358146815781F70164807580BC
:10A0E00086809780C601861B970B97FDD8C0809706
:10A0F0000CF46CC06C157D050CF0ADC066247724A3
:10A100004301F8016181F7018181681709F499C061
:10A11000662309F491C0621A730A840A950AA4019D
:10A12000930157FDC0C0F5011182B60119012A0142
:10A1300079018A0139014A0108946108710881088E
:10A140009108FFEF6F16FFEF7F06FFEF8F06FFE32B
:10A150009F06F0F4A8019701220F331F441F551FDB
:10A1600019012A01B601615070406B0179018A0121
:10A1700039014A01089461087108810891088FEF3C
:10A1800068168FEF78068FEF88068FE3980610F336
:10A1900083E0D5018C9357FC64C0F501248335839B
:10A1A0004683578373836283A50189C06F5F7F4FA6
:10A1B000D401C30181709070A070B07096948794A0
:10A1C00077946794682A792A8A2A9B2A6C157D05D8
:10A1D0006CF311C00894C11CD11CDA01C901817053
:10A1E0009070A070B0705695479537952795282B9D
:10A1F000392B4A2B5B2BC616D70664F382CFF801A6
:10A200009181FB018181981709F453CF41E751E017
:10A2100056C0823009F04DCF88E0DA01F801019094
:10A220000D928A95E1F7F8018181FB0191818923E3
:10A23000FA018183A50143C0261937094809590944
:10A2400070CFF5016183B601260D371D481D591DDC
:10A2500019012A019DCF6B0120E030E040E050E081
:10A2600050CFD201C101B695A7959795879521E06A
:10A2700030E040E050E02222332244225522282AB6
:10A28000392A4A2A5B2AF50124823582468257827E
:10A290000894C11CD11CD382C282A50110C0909524
:10A2A00081959F4F24CF81E0F5018183B6015095C0
:10A2B0004095309521953F4F4F4F5F4F37CFCA01A3
:10A2C000E2E1CDB7DEB70C941956A0E2B0E0EBE6C0
:10A2D000F1E50C940B56DC01CB01898F9A8FAB8F83
:10A2E000BC8F2D8F3E8F4F8F58A3BE016F5F7F4F66
:10A2F000CE0149960E944F548E01075F1F4FB8014F
:10A30000CE014D960E944F54AE014F5E5F4FB80193
:10A31000CE0101960E9441500E946753DC01CB019F
:10A32000BC01CD01E4E0A0960C942756A0E2B0E079
:10A33000ECE9F1E50C940B56DC01CB01898F9A8F87
:10A34000AB8FBC8F2D8F3E8F4F8F58A3BE016F5F99
:10A350007F4FCE0149960E944F548E01075F1F4FD9
:10A36000B801CE014D960E944F548A8591E089270D
:10A370008A87AE014F5E5F4FB801CE0101960E9401
:10A3800041500E946753DC01CB01BC01CD01E4E0E8
:10A39000A0960C942756A8E1B0E0E1EDF1E50C940D
:10A3A0000556DC01CB01898B9A8BAB8BBC8B2D8B3B
:10A3B0003E8B4F8B588FBE016F5F7F4FCE01419612
:10A3C0000E944F548E01075F1F4FB801CE01459682
:10A3D0000E944F54FE0131962981223008F45FC05B
:10A3E0003985323010F4B8017BC081819A85892784
:10A3F0008183243009F455C0223009F452C034302E
:10A4000009F454C0323009F458C06B817C818B85CB
:10A410009C85681B790B2D813E814F815885ED8489
:10A42000FE840F8518892E153F054007510730F42B
:10A43000220F331F441F551F615070407C836B8374
:10A4400080E090E0A0E0B0E4AA24BB2465012E15D2
:10A450003F054007510740F0A82AB92ACA2ADB2A3B
:10A460002E193F09400B510BB695A79597958795E7
:10A47000220F331F441F551F0097A105B10539F75F
:10A48000D601C5018F779070A070B07080349105AF
:10A49000A105B105A9F0A482B582C682D782BF0109
:10A4A0001FC02317E1F761E771E01AC01D821E8209
:10A4B0001F8218861C821B82F2CF84E08983EFCF33
:10A4C000A7FC05C0211531054105510521F380E4A4
:10A4D00090E0A0E0B0E0A80EB91ECA1EDB1EDBCFE4
:10A4E000CB010E946753DC01CB01BC01CD01EAE046
:10A4F00068960C942156A8E1B0E0E1E8F2E50C94EE
:10A500000B56DC01CB01898B9A8BAB8BBC8B2D8BD3
:10A510003E8B4F8B588FBE016F5F7F4FCE014196B0
:10A520000E944F548E01075F1F4FB801CE01459620
:10A530000E944F548981823018F08985823018F446
:10A540002FEF3FEF09C0B801CE0101960E94C95418
:10A55000282F332727FD3095C901E4E068960C9435
:10A560002756A8E0B0E0E7EBF2E50C9409569B0112
:10A57000AC017B018C01EE2417FDE394FF2400273E
:10A580001127EA82211531054105510539F482E090
:10A590008983CE0101960E94675343C083E089837B
:10A5A0006EE170E0CB01EE2031F579018A01A8015E
:10A5B00097012030E0E03E07E0E04E07E0E45E0770
:10A5C00098F479018A01EE0CFF1C001F111F0197FE
:10A5D000BC01A8019701E0E0EE16E0E0FE06E0E035
:10A5E0000E07E0E41E0768F3ED82FE820F831887F2
:10A5F0007C836B83CECF2030E0E03E07E0E04E0767
:10A60000E0E85E0741F0EE24FF248701E21AF30A36
:10A61000040B150BCCCF7C836B8360E070E080E093
:10A620009FECE6E028960C942556ACE0B0E0EBE118
:10A63000F3E50C940D56DC01CB0189879A87AB8733
:10A64000BC87BE016F5F7F4FCE0109960E944F54B9
:10A650008981823011F0823028F460E070E080E07F
:10A6600090E031C0843039F02B813C8137FDF5CF4B
:10A670002F3131056CF08A81882329F060E070E089
:10A6800080E090E820C06FEF7FEF8FEF9FE71BC067
:10A690008EE190E0821B930B2D813E814F81588586
:10A6A00004C056954795379527958A95D2F78A81A4
:10A6B000882339F050954095309521953F4F4F4F65
:10A6C0005F4FCA01B901E2E02C960C942956A0E034
:10A6D000B0E0EDE6F3E50C94035688249924540188
:10A6E000DC01FC0124813581468157818181082F5D
:10A6F000112760E070E08C91823020F46FEF70E001
:10A700004061A4C0843009F464C0823009F463C09D
:10A71000211531054105510509F498C0FD018281DB
:10A720009381FFEF82389F070CF050C0A2E8EA2E19
:10A73000AFEFFA2EE81AF90A8AE1E816F1040CF0F4
:10A740006BC06B0181E090E0A0E0B0E00E2C04C093
:10A75000880F991FAA1FBB1F0A94D2F70197A1095E
:10A76000B10982239323A423B5230097A105B10542
:10A7700019F0F1E0CF2ED12C04C0569547953795AE
:10A780002795EA94D2F7C601AA2797FDA095BA2F7C
:10A79000282B392B4A2B5B2BDA01C9018F7790705C
:10A7A000A070B07080349105A105B105D1F1215C94
:10A7B0003F4F4F4F5F4F2030E0E03E07E0E04E0755
:10A7C000E0E45E0708F161E070E01EC080389105AA
:10A7D0003CF06FEF70E020E030E040E050E036C049
:10A7E000BC0161587F4FDA01C9018F779070A0706A
:10A7F000B07080349105A105B105D1F0215C3F4FC7
:10A800004F4F5F4F57FD1BC097E0569547953795C3
:10A8100027959A95D1F71AC020E030E040E050E04B
:10A82000BBCF27FFC8CF205C3F4F4F4F5F4FC3CFF9
:10A8300027FFE8CF205C3F4F4F4F5F4FE3CF569548
:10A840004795379527956F5F7F4FDECF822E932EEA
:10A85000942F9F778A2D8078A82EA92A962F9795D6
:10A86000992797958A2D8F77A82EA92A769567958F
:10A87000962F9F778B2D8078B82EB92A902F979599
:10A88000992797958B2D8F77B82EB92AD501C401BA
:10A89000BC01CD01ECE0CDB7DEB70C941F56CF93D1
:10A8A000DF93FC01DB01408151812281622F6F77B0
:10A8B00070E0221F2227221F9381892F880F822B6D
:10A8C000282F3327991F9927991FED019983211567
:10A8D000310541F44115510561057105E1F482E04E
:10A8E0008C9354C02F3F310509F441C02F5730409D
:10A8F000FD013383228383E08C9387E0440F551F4F
:10A90000661F771F8A95D1F77064ED014C835D83D4
:10A910006E837F833BC022E83FEFF901C7E0440F1D
:10A92000551F661F771FCA95D1F783E08C9340307F
:10A9300080E0580780E0680780E4780778F4440FE7
:10A94000551F661F771F21503040F9014030C0E08D
:10A950005C07C0E06C07C0E47C0788F3ED01FB8373
:10A96000EA83FD0144835583668377830FC04115D5
:10A9700051056105710519F484E08C9307C064FFEB
:10A9800003C081E08C93C1CF1C92BFCFDF91CF91E8
:10A9900008950F931F93CF93DF93FC01DB01808118
:10A9A000823018F09C91923018F461E070E05EC043
:10A9B0008430C1F0843001F1943009F447C0823012
:10A9C00009F44BC0823009F44EC09230A9F04181A5
:10A9D000ED0189814817B9F0442389F08FEF9FEF8B
:10A9E000BC0144C0943031F7EB018981682F77278F
:10A9F0008181681B71093AC08181882379F781E0E0
:10AA000090E0BC0133C022813381ED018A819B81BA
:10AA1000821793070CF3281739079CF004811581DE
:10AA200026813781FD016481758186819781601758
:10AA300071078207930780F206171707280739075F
:10AA400078F4442359F281E090E0DBCFFD0181816D
:10AA5000882321F281E090E0D4CF923009F0B2CF88
:10AA600060E070E003C0ED018981F2CFCB01DF919E
:10AA7000CF911F910F910895FB01DC0105900D927C
:10AA80000020E1F70895FB01DC0104C08D910190E5
:10AA9000801921F441505040C8F7881B990B089544
:10AAA000FB01DC0140FF05C002C001900D92019046
:10AAB0000D9242505040C8F70895DC0140FF03C09A
:10AAC00001C06D936D9342505040D8F70895FB013B
:10AAD000DC0101900D920020E1F70895629FD00102
:10AAE000739FF001829FE00DF11D649FE00DF11D49
:10AAF000929FF00D839FF00D749FF00D659FF00DF8
:10AB00009927729FB00DE11DF91F639FB00DE11DE4
:10AB1000F91FBD01CF0111240895991B79E004C0EC
:10AB2000991F961708F0961B881F7A95C9F780958C
:10AB30000895AA1BBB1B51E107C0AA1FBB1FA61784
:10AB4000B70710F0A61BB70B881F991F5A95A9F7D6
:10AB500080959095BC01CD01089597FB092E07269D
:10AB60000AD077FD04D0E5DF06D000201AF47095F6
:10AB700061957F4F0895F6F7909581959F4F0895C1
:10AB8000A1E21A2EAA1BBB1BFD010DC0AA1FBB1FF1
:10AB9000EE1FFF1FA217B307E407F50720F0A21B63
:10ABA000B30BE40BF50B661F771F881F991F1A94D0
:10ABB00069F760957095809590959B01AC01BD01FA
:10ABC000CF01089597FB092E05260ED057FD04D01E
:10ABD000D7DF0AD0001C38F4509540953095219568
:10ABE0003F4F4F4F5F4F0895F6F7909580957095C2
:10ABF00061957F4F8F4F9F4F08952F923F924F92B5
:10AC00005F926F927F928F929F92AF92BF92CF92FC
:10AC1000DF92EF92FF920F931F93CF93DF93CDB705
:10AC2000DEB7CA1BDB0B0FB6F894DEBF0FBECDBF7D
:10AC300009942A88398848885F846E847D848C844E
:10AC40009B84AA84B984C884DF80EE80FD800C8157
:10AC50001B81AA81B981CE0FD11D0FB6F894DEBF3A
:10AC60000FBECDBFED010895F999FECFB2BDA1BDD4
:10AC7000F89A119600B40895F7DF01921A94E1F75B
:10AC80000895F999FECFB2BDA1BD00BC11960FB6D3
:10AC9000F894FA9AF99A0FBE08950190F2DF1A9487
:04ACA000E1F708953B
:10ACA40001012E2E2F63616E5F696E7075742E63C1
:10ACB400006E2E2E2F6368616E6E656C732E6300BA
:10ACC400455233002E2E2F656570726F6D63686177
:10ACD4006E6E656C732E630050434D3000455233E5
:10ACE400004C4F4730340050434D20766572203875
:10ACF4002E3037004F425220383434300B002E2E81
:10AD04002F7669727475656C5F696E7075742E63E5
:0AAD14000000000000000000000035
:00000001FF
